:020000020000FC
:0200000024C01A
:02003C00F6C00C
:1000480008C100E10EBF0FEF0DBF010F60D79CD0B4
:1000580067D073D08CD07ED007E003BF02E007BF23
:1000680033240FEFF02E0093D9093092D209ECEF28
:10007800FFEFA191B08107E40FE40091FFFF009129
:10008800FFFF009100E00091FEFF10E4FF27E5EC80
:10009800F13130F00F2F007F003859F0108309C07C
:1000A80002E000936C00F0641083FF7B00E0009393
:1000B8006C00EBECF13130F00F2F007F003859F075
:1000C800108309C002E000936C00F0641083FF7B8A
:1000D80000E000936C000FB7D02E789400270091B1
:1000E800D20901FDF0D0ECE8F0E1B13110F08D91CA
:1000F80009C002E000936C00B0648D91BF7B00E002
:1001080000936C000027880F031DE80FF01FC591AE
:10011800D491FE01F8940994000000000000E5CF96
:10012800ECE8F2E1C0E0D0EE002710E22591299337
:100138001A95E1F70A95C9F70895ECE8F2E3C0E0EB
:10014800D0EC002710E2259129931A95E1F70A953A
:10015800C9F70895ECE8F2E6C0E0D0EA002710E21B
:10016800259129931A95E1F70A95C9F70895ECE8BE
:10017800F2E5C0E0D0E8002710E1259129931A950F
:10018800E1F70A95C9F70895ECE8F2E5C0E0D0E890
:1001980011E006E477D6112700E074D600EF72D696
:1001A80011E002E46FD61127332720E105916AD6C2
:1001B8002A95E1F73A95C9F708950F921F920F9380
:1001C8001F932F933F934F93EF93FF93E0E0F0E15A
:1001D80036E147E1CC24BB24F1D5FBD511E002E49C
:1001E80051D61127F13110F0219109C002E0009396
:1001F8006C00F0642191FF7B00E000936C00022FFB
:1002080041D6B394B31671F7C394C41621F7FF917E
:10021800EF914F913F912F911F910F911F900F9048
:1002280008951F921FB60F931F930091D20900FFE4
:1002380002C00E7F01C0016000FFBFDF1E2D0D7FD1
:1002480017FF02600093D2091F910F911FBE1F90E4
:1002580018951F921FB60F931F93EF93FF931CB12E
:10026800E7E7F2E0F13130F00F2F007F003859F066
:10027800108309C002E000936C00F0641083FF7BD8
:1002880000E000936C0011E0E6ECF0E0F13130F0B2
:100298000F2F007F003859F0108309C002E0009347
:1002A8006C00F0641083FF7B00E000936C00FF910A
:1002B800EF911F910F911FBE1F9018955D9BFECF68
:1002C8000CB959D00895F1E0EF2D02E000936C00CD
:1002D800F064B083FF7B00E000936C00FA94F1E0D7
:1002E800EF2D02E000936C00F064A083FF7B00E038
:1002F80000936C00FA9449D5F1E0EF2D02E00093E9
:100308006C00F0648083FF7B00E000936C00FA943B
:100318000E2D0068E02E0091D2090D7F0093D209BE
:10032800CEEFDFEFA991B88108951F932F933F93E4
:10033800E13229F080813F912F911F9108958FEF2D
:100348001091D9091F3FB9F3212F26952695269597
:1003580030912091222319F036952A95FBCF30FF52
:1003680001C0E9CF17708EEF112321F00894881F80
:100378001A95FACFE0CF3F932F9324E135E83A95C9
:10038800000000000000D9F72A95C1F72F913F918E
:1003980008952F9324E6EFDF2A95E9F72F91089522
:1003A80034D3DFBE582BDFB698CE2FD3DFBE582309
:1003B800DFB693CE2AD3DFBE5827DFB68ECE25D33D
:1003C800DFBE11E0581F0FB7D02E1E2D03FF1F7B75
:1003D80003FD1064E12E81CE18D3852FF13130F062
:1003E8000F2F007F003859F0508309C002E00093B6
:1003F8006C00F0645083FF7B00E000936C006DCECE
:1004080004D3582F1D2D55230FB702FF1B7F02FD64
:10041800146001FF1D7F01FD1260D12E5ECEF5D262
:10042800581710F0089401C08894DFB656CEEDD264
:10043800DFBE10F0089401C088941894580B10F08F
:10044800089401C08894DFB60FB71E2D03FF1F7BE9
:1004580003FD1064E12E41CEE9D2880FDFB6F131F9
:1004680030F00F2F007F003859F0808309C002E078
:1004780000936C00F0648083FF7B00E000936C00C5
:100488002CCED4D2DFBE881FDFB6F13130F00F2F6B
:10049800007F003859F0808309C002E000936C00A7
:1004A800F0648083FF7B00E000936C0016CEBED220
:1004B8008695DFB6F13130F00F2F007F003859F004
:1004C800808309C002E000936C00F0648083FF7BA6
:1004D80000E000936C0001CEA9D2DFBE8795DFB69D
:1004E800F13130F00F2F007F003859F0808309C0B8
:1004F80002E000936C00F0648083FF7B00E00093CF
:100508006C00EBCD93D2862FF13130F00F2F007FA6
:10051800003859F0808309C002E000936C00F06451
:100528008083FF7B00E000936C00D7CD7FD2682FDB
:100538001D2D66230FB702FF1B7F02FD146001FF0C
:100548001D7F01FD1260D12EC8CD70D2DFBE8A9505
:10055800DFB6F13130F00F2F007F003859F080837B
:1005680009C002E000936C00F0648083FF7B00E028
:1005780000936C00B2CD5AD2DFBE8395DFB6F1315D
:1005880030F00F2F007F003859F0808309C002E057
:1005980000936C00F0648083FF7B00E000936C00A4
:1005A8009CCD44D2DFBE052F08230FB787FF0B7FF2
:1005B80087FD0460D02E0E2D86FF0F7B86FD00641C
:1005C800E02E8BCDB13110F02D9109C002E00093DF
:1005D8006C00B0642D91BF7B00E000936C00B131DA
:1005E80010F01D9109C002E000936C00B0641D91E9
:1005F800BF7B00E000936C00A22FB12F6ECDB1310C
:1006080010F0CD9109C002E000936C00B064CD9168
:10061800BF7B00E000936C00B13110F0DD9109C0A0
:1006280002E000936C00B064DD91BF7B00E00093B2
:100638006C00D13110F0A88109C002E000936C0071
:10064800D064A881DF7B00E000936C00C395D131B2
:1006580010F0B88109C002E000936C00D064B88142
:10066800DF7B00E000936C0038CDE0D1872FF131BB
:1006780030F00F2F007F003859F0808309C002E066
:1006880000936C00F0648083FF7B00E000936C00B3
:1006980024CDCCD1782F1D2D77230FB702FF1B7FD8
:1006A80002FD146001FF1D7F01FD1260D12E15CDE2
:1006B800BDD1781710F0089401C08894DFB60DCD2D
:1006C800B5D1681710F0089401C08894DFB605CD3D
:1006D8000D2D02FF46C3119600CD0D2D02FD41C31D
:1006E8001196FBCC0E2D06FF3CC31196F6CC0E2DB1
:1006F80006FD37C31196F1CC0D2D00FF32C31196BC
:10070800ECCC0D2D00FD2DC31196E7CC0D2D01FF6E
:1007180028C31196E2CC0D2D01FD23C31196DDCC23
:1007280002E4CCDD00000000D8CCB13110F01D91FE
:1007380009C002E000936C00B0641D91BF7B00E02B
:1007480000936C00F1E0EF2D02E000936C00F06480
:10075800B083FF7B00E000936C00FA94F1E0EF2D8A
:1007680002E000936C00F064A083FF7B00E000933C
:100778006C00FA94B13110F02D9109C002E0009399
:100788006C00B0642D91BF7B00E000936C00A12F3A
:10079800B22FA3CCF394F1E0EF2D02E000936C00AC
:1007A800F0648081FF7B00E000936C00F5D2F39445
:1007B800F1E0EF2D02E000936C00F064A081FF7B74
:1007C80000E000936C00F394F1E0EF2D02E0009359
:1007D8006C00F064B081FF7B00E000936C000000C7
:1007E80000007BCCF394F1E0EF2D02E000936C0065
:1007F800F064A081FF7B00E000936C00F394F1E0CB
:10080800EF2D02E000936C00F064B081FF7B00E004
:1008180000936C00119661CC550FDFB65ECCDFBE3D
:10082800551FDFB65ACC5695DFB657CCDFBE579565
:10083800DFB653CC10D2862FF13130F00F2F007F66
:10084800003859F0808309C002E000936C00F0641E
:100858008083FF7B00E000936C003FCCFCD1682FC5
:100868001D2D66230FB702FF1B7F02FD146001FFD9
:100878001D7F01FD1260D12E30CC11D2682F1D2DA5
:1008880066230FB702FF1B7F02FD146001FF1D7F67
:1008980001FD1260D12E21CC78D2F1E0EF2D02E0DB
:1008A80000936C00F0648083FF7B00E000936C0091
:1008B800FA9413CCF394F1E0EF2D02E000936C006E
:1008C800F0648081FF7B00E000936C0065D205CC6A
:1008D800F1E0EF2D02E000936C00F0645083FF7BA1
:1008E80000E000936C00FA94F8CBF394F1E0EF2D5C
:1008F80002E000936C00F0645081FF7B00E00093FD
:100908006C001D2D55230FB702FF1B7F02FD1460DD
:1009180001FF1D7F01FD1260D12EDFCBDFBE7A956E
:10092800DFB6DBCB752F1D2D77230FB702FF1B7F9B
:1009380002FD146001FF1D7F01FD1260D12ECDCB99
:10094800DFBE7395DFB6C9CBDFBE6395DFB6C5CB17
:100958000D2D0E7FD02EC1CB0D2D0160D02EBDCB1D
:100968000E2D0F77E02EB9CB0E2D0068E02EB5CBFB
:10097800572F1D2D55230FB702FF1B7F02FD146053
:1009880001FF1D7F01FD1260D12EA7CB0E2D0F7B1D
:10099800E02EA3CB0E2D077FE02E9FCB0E2D0860F7
:1009A800E02E9BCB562F1D2D55230FB702FF1B7F23
:1009B80002FD146001FF1D7F01FD1260D12E8DCB59
:1009C800F62E8BCB652F1D2D66230FB702FF1B7FDD
:1009D80002FD146001FF1D7F01FD1260D12E7DCB49
:1009E8006F2D1D2D66230FB702FF1B7F02FD1460BC
:1009F80001FF1D7F01FD1260D12E6FCBDFBE6A950E
:100A0800DFB66BCB0000000068CB88738030D9F06C
:100A18008830D1F08031C9F08831C1F08032B9F026
:100A28008832B1F08033B1F08833A9F08873803010
:100A380061F0883049F0803179F0883139F08832B6
:100A480039F0883341F009C046C067C074C0A1C0FE
:100A5800DEC001C124C153C182C1D0E0B13110F060
:100A6800CD9109C002E000936C00B064CD91BF7BCA
:100A780000E000936C00C60FD31DD13110F0E9914E
:100A880009C002E000936C00D064E991DF7B00E0CC
:100A980000936C00D13110F0F88109C002E0009396
:100AA8006C00D064F881DF7B00E000936C000F2FAE
:100AB800013971F0F13110F080810CC002E000932F
:100AC8006C00F0648081FF7B00E000936C0002C042
:100AD8002CDC882F0895F0E0B13110F0ED9109C0B9
:100AE80002E000936C00B064ED91BF7B00E00093DE
:100AF8006C000F2F013971F0F13110F080810CC0BA
:100B080002E000936C00F0648081FF7B00E00093BA
:100B18006C0002C00ADC882F0895B13110F08D9165
:100B280009C002E000936C00B0648D91BF7B00E0C7
:100B380000936C000895B13110F0ED9109C002E006
:100B480000936C00B064ED91BF7B00E000936C00F3
:100B5800B13110F0FD9109C002E000936C00B0645F
:100B6800FD91BF7B00E000936C000F2F013971F0FD
:100B7800F13110F080810CC002E000936C00F06449
:100B88008081FF7B00E000936C0002C0CEDB882FE1
:100B98000895D0E0B13110F0CD9109C002E0009382
:100BA8006C00B064CD91BF7B00E000936C00D13144
:100BB80010F0E99109C002E000936C00D064E9915B
:100BC800DF7B00E000936C00D13110F0F88109C0A0
:100BD80002E000936C00D064F881DF7B00E00093B2
:100BE8006C00E70FF31D0F2F013971F0F13110F090
:100BF80080810CC002E000936C00F0648081FF7B70
:100C080000E000936C0002C090DB882F0895F0E0AC
:100C1800B13110F0ED9109C002E000936C00B064AE
:100C2800ED91BF7B00E000936C00E60FF31D0F2FE2
:100C3800013971F0F13110F080810CC002E00093AD
:100C48006C00F0648081FF7B00E000936C0002C0C0
:100C58006CDB882F0895F0E0B13110F0ED9109C0F8
:100C680002E000936C00B064ED91BF7B00E000935C
:100C78006C00E70FF31D0F2F013971F0F13110F0FF
:100C880080810CC002E000936C00F0648081FF7BDF
:100C980000E000936C0002C048DB882F0895B13152
:100CA80010F0ED9109C002E000936C00B064ED9182
:100CB800BF7B00E000936C00B13110F0FD9109C0DA
:100CC80002E000936C00B064FD91BF7B00E00093EC
:100CD8006C00E70FF31D0F2F013971F0F13110F09F
:100CE80080810CC002E000936C00F0648081FF7B7F
:100CF80000E000936C0002C018DB882F0895B13122
:100D080010F0ED9109C002E000936C00B064ED9121
:100D1800BF7B00E000936C00B13110F0FD9109C079
:100D280002E000936C00B064FD91BF7B00E000938B
:100D38006C00E60FF31D0F2F013971F0F13110F03F
:100D480080810CC002E000936C00F0648081FF7B1E
:100D580000E000936C0002C0E8DA882F0895852F20
:100D68000895B13110F02D9109C002E000936C0094
:100D7800B0642D91BF7B00E000936C0027FD1FEF4E
:100D880027FF10E0A20FB11FA8C90D2D07701E2D57
:100D9800187F012B802F0895D82EE82E089506E598
:100DA8008DDA9BC9FFCF5F9BFECF1CB15F9BFECF47
:100DB8000CB168D05D9BFECF0CB9F5CF0F931F9394
:100DC8000C2D10E5109F11270B0C111E1F910F9170
:100DD80008951F930F930092D0091092D10911E042
:100DE80006E450D01127002D4DD0012D4BD00F9186
:100DF8001F9108950F931F932F93EF93FF93202F25
:100E080011E002E43FD01127022F3CD00091D00915
:100E18001091D109E0E0F2E0E00FF11F21932227C1
:100E28000395121F0093D0091093D109FF91EF91F8
:100E38002F911F910F9108950F921F920F931F9357
:100E48002F93EF93FF93BADFC4DF202F11E002E462
:100E580019D01127022F16D0002D112DE0E0F2E055
:100E6800E00FF11F219322270395121F0093D00949
:100E78001093D109FF91EF912F911F910F911F901E
:100E88000F9008951F930F931E9810FF1F9810FD41
:100E98001F9A08BB00000000000000001D98000019
:100EA800000000001D9A000000001E9A0F911F917B
:100EB80008950F9300270861009365005CDA002706
:100EC80008600093650057DA0F9108950F93002783
:100ED8000861009365004FDA002700610093650000
:100EE8004ADA002708610093650045DA00270860A0
:100EF8000093650040DA0F9108953DDA97983BDA40
:100F0800979A39DA38DA37DA36DA35DA089508E0CE
:100F18000093650008E1009364000FEF07BB00E051
:100F280008BB179A159A149A169A8F9A979A1F9827
:100F38001F9A1D9A1C9A1E9800EC05BF01E00093A9
:100F48006D000FEF04BB00E005BB00E00AB90BB968
:100F580008E90AB900E109B9AA249924BB24CC24D8
:100F680000270093D0090093D10905DAC6DF03DA18
:100F7800ADDF01DA1E98FFD91E9A0FE19ADF0A95B4
:100F8800E9F726D001D008950F931F932F933F932D
:100F9800EF93FF93E0E0F2E011E002E473DF112742
:100FA80039E120E500E26EDF11932A95D9F73A95E9
:100FB800C1F711E006E466DF112700E063DF00E017
:100FC80061DFFF91EF913F912F911F910F9108954C
:100FD80011E000E457DF112701E354DF07E852DF8F
:100FE80007E050DF07E24EDF0FE24CDF07EC4ADF95
:100FF80000E548DF00E046DF11E00CE543DF11279C
:1010080000E040DF00EF3EDF11E004E43BDF1127A2
:1010180000E038DF00E036DF07EC34DF00E032DFE5
:1010280005E030DF07EC2EDF00E02CDF00E02ADFF0
:1010380000E028DF00E026DF11E00AE523DF1127C2
:1010480000E020DF11E006E41DDF112700E01ADFD1
:1010580000E018DF11E00BE515DF112700E012DFD3
:1010680011E00DE50FDF112707E00CDF07E80ADFC5
:1010780011E00CE407DF11E009E504DF112706E0C1
:1010880001DF08959403D4013002D306D306D401B6
:101098003002D3065004D4011004D306D306D40179
:1010A8003002D3066C03D4013002D306D306D40130
:1010B8003002D306AC04D4013002D306D306D401DF
:1010C8003002D3069903D9014502D306D502D901C6
:1010D8004502D3065E04D9011304D306D502D9010B
:1010E8004502D3067103D9014502D306D502D901B9
:1010F8004502D306B004D9014502D306D502D90169
:101108004502D306CE03DE015B02D306E602DE010A
:101118005B02D3066C04DE011704D306E602DE0187
:101128005B02D3067603DE015B02D306E602DE012C
:101138005B02D306B404DE015B02D306E602DE01DD
:101148005B02D306F603E3017002D3060303E3014F
:101158007002D3067904E3011A04D3060303E301FA
:101168007002D3067B03E3017002D3060303E30195
:101178007002D306B804E3017002D3060303E30147
:101188007002D3063903F0018602D3063903F00151
:101198008602D3069204F001D604D3063903F0017F
:1011A8008602D3068003F0018602D3063903F001D4
:1011B8001E04D306BC04F001E404D3063903F0018D
:1011C8008602D3064D0304029A02D3064D03040295
:1011D8009A02D30696040402E604D3064D030402D9
:1011E8009A02D306850304029A02D3064D03040229
:1011F8003204D306CA040402F404D3064D030402DD
:101208004104D3065C031302A902D3065C0313024C
:10121800A902D306A40413020205D3065C03130231
:10122800A902D3068A031302A902D3065C03130298
:10123800A902D306CE041302A902D3065C03130243
:10124800A902D30664031B02BF02D30664031B0270
:10125800BF02D306A8041B020605D30664031B02BB
:10126800BF02D3068F031B02BF02D30664031B020F
:10127800BF02D306D2041B02BF02D30664031B02BB
:10128800BF02D3060FDCA561C988900320D4DA20F9
:10129800CCDCA507186981F0F338E90148A205B547
:1012A80069B46195619469CA10F5A5568570205393
:1012B800D820B4DFA9C4A0DF2056E0A900856F6854
:1012C80020B9DA608571847220CADBA9572028DA30
:1012D800205AE0A957A0004C28DA8571847220C7EB
:1012E800DBB1718567A471C898D002E6728571A4D4
:1012F800722028DAA571A4721869059001C8857151
:1013080084722067D8A95CA000C667D0E4609835CD
:10131800447A006828B14600202BDC3037D02020E2
:10132800F3FF86228423A004B1228562C8B12285F6
:1013380064A008B1228563C8B12285654CE0E0A9A4
:101348008BA00020A2DBA98AA0E02028DAA98FA020
:10135800E02067D8A665A56285658662A663A56450
:1013680085638664A9008566A5618570A980856105
:1013780020D7D8A28BA0004CD4DBC9F0D007843882
:1013880086374C63C6AAD002A21E4C37C420D2FFAF
:10139800B0E86020CFFFB0E26020C9FFB0DC602079
:1013A800C6FFB0D66020E4FFB0D060208ACD20F719
:1013B800D7A9E148A94348AD0F0348AD0C03AE0DCA
:1013C80003AC0E03286C1400088D0C038E0D038CDF
:1013D8000E03688D0F036020D1E1A62DA42EA92B42
:1013E80020D8FFB09560A9012CA900850A20D1E179
:1013F800A50AA62BA42C20D5FFB057A50AF01AA23F
:101408001C20B7FF2910F0034C37C4A57AC902F095
:1014180007A964A0C34C1ECB6020B7FF29BFF00505
:10142800A21D4C37C4A57BC902D00E862D842EA9D7
:1014380076A0C3201ECB4C2AC5208EC64C76E4204D
:1014480016E220C0FFB00B602016E2A54920C3FFBA
:1014580090C64CF6E0A90020BDFFA201A00020BA6A
:10146800FF2003E22054E22003E220FDE1A00086F1
:101478004920BAFF2003E220FDE18AA8A6494CBA18
:10148800FF200BE24C9ED7207900D00268686020CC
:10149800FDCE207900D0F74C08CFA90020BDFF2051
:1014A8000EE2209ED786498AA201A00020BAFF201A
:1014B80003E220FDE1864AA000A549E003900188E7
:1014C80020BAFF2003E220FDE18AA8A64AA5492008
:1014D800BAFF2003E2200BE2209ECD20A3D6A6224D
:1014E800A4234CBDFFA9DDA0E22067D8200CDCA90D
:1014F800E2A0E2A66E2007DB200CDC20CCDCA900F1
:10150800856F2053D8A9E7A0E22050D8A5664810D7
:101518000D2049D8A5663009A51249FF851220B4C7
:10152800DFA9E7A0E22067D868100320B4DFA9ECA0
:10153800A0E24C40E020CADBA90085122068E2A2A4
:101548004EA00020F3E0A957A00020A2DBA9008547
:1015580066A51220D9E2A94EA0004C0FDB484C9A90
:10156800E281490FDAA283490FDAA27F0000000066
:101578000584E61A2D1B862807FBF88799688901D8
:10158800872335DFE186A55DE72883490FDAA2A521
:101598006648100320B4DFA56148C9819007A9BC3B
:1015A800A0D9200FDBA93BA0E32040E068C98190C7
:1015B80007A9DDA0E22050D86810034CB4DF600B07
:1015C80076B383BDD3791EF4A6F57B83FCB0107C7B
:1015D8000C1F67CA7CDE53CBC17D1464704C7DB789
:1015E800EA517A7D6330887E7E9244993A7E4CCC6B
:1015F80091C77FAAAAAA138100000000205BE420FB
:10160800A4E32004E4A2FB9A4C74C4E67AD002E670
:101618007BAD60EAC93AB00AC920F0EF38E9303842
:10162800E9D060804FC75258A94C85548500A94815
:10163800A0D285018402A991A0D385058406A9AA10
:10164800A0D185038404A21CBD87E39573CA10F852
:10165800A9038553A900856885138518A2018EFD05
:10166800018EFC01A219861638209CFF862B842C3B
:10167800382099FF8637843886338434A0009891BF
:101688002BE62BD002E62C60A52BA42C2008C4A99D
:1016980036A0E4201ECBA53738E52BAAA538E52CC3
:1016A80020CDDDA929A0E4201ECB4C44C6204259F8
:1016B80054455320465245450D00932A2A2A2A208C
:1016C80043424D204241534943205632202A2A2A78
:1016D8002A0D003AC483C47CC51AC7E4C786CEA2C3
:1016E8000BBD4FE49D0003CA10F76020CCFFA90092
:1016F8008513207AC6584C74C4412033C54C77C62C
:10170800FFFFFFFFFFFFFFFFFFFFFFFFFFFFFFFFE1
:10171800FFFFFFFFFFFFFFFFFFFFFFFFFFFFFFFFD1
:10172800FFFFFFFFAD2C9129DF8D2C9160AD2C912F
:1017380009208D2C9160AD1F91CD1F91D0F84A6082
:10174800A6B94C47F68AD008A5C385AEA5C485AF0F
:101758004C6AF620E3F8900368A9004C9EF3FFFF5B
:10176800FFFFFFFFFFFFFFFFFFFFFFFFFFFFFFFF81
:10177800FFFFFFFFFFFFFFFFFFFFFFFFFFFFFFFF71
:10178800FFFFFFFFA210A09160A216A01760B0078C
:1017980086D684D32087E5A6D6A4D36020BBE5AD42
:1017A800880229FD0A0A09808D0590AD8802290260
:1017B800F008A9800D02908D0290A9008D910285F4
:1017C800CFA9DC8D8F02A9EB8D9002A90A8D890221
:1017D8008D8C02A9068D8602A9048D8B02A90C8521
:1017E800CD85CCAD88020980A8A900AA94D918692A
:1017F800169001C8E8E018D0F3A9FF95D9A21620E1
:101808008DEACA10FAA00084D384D6A6D6A5D3B48C
:10181800D9300818691685D3CA10F4B5D929030D2B
:10182800880285D2BDFDED85D1A915E8B4D9300669
:10183800186916E810F685D56020BBE54C81E5A946
:1018480003859AA9008599A210BDE3ED9DFF8FCA73
:10185800D0F760AC7702A200BD78029D7702E8E479
:10186800C6D0F5C6C6985818602042E7A5C685CCEC
:101878008D9202F0F778A5CFF00CA5CEAE8702A026
:101888000084CF20A1EA20CFE5C983D010A209782F
:1018980086C6BDF3ED9D7602CAD0F7F0CFC90DD04C
:1018A800C8A4D584D0B1D1C920D00388D0F7C884C2
:1018B800C8A0008C920284D384D4A5C9301DA6D6B2
:1018C8002019E7E4C9D014D012A5CA85D3C5C89099
:1018D8000AB04298488A48A5D0F091A4D3B1D1EA79
:1018E800EAEAEAEAEAEAEAEAEAEAEAEAEAEAEAEA50
:1018F800EAEAEAEAEAEA85D7293F06D724D71002B6
:1019080009809004A6D4D00470020940E6D320B818
:10191800E6C4C8D017A90085D0A90DA699E003F0A0
:1019280006A69AE003F0032042E7A90D85D768AA26
:1019380068A8A5D7C9DED002A9FF1860C922D008B7
:10194800A5D4490185D4A922600940A6C7F0020997
:1019580080A6D8F002C6D8AE860220A1EA20EAE620
:1019680068A8A5D8F00246D468AA6818586020FA72
:10197800E8E6D3A5D5C5D3B037C957F02AAD92024A
:10198800F0034CF0E9A6D6E01790072075E9C6D613
:10199800A6D616D956D94C5BED691685D5B5D9307A
:1019A80003CAD0F94C7EEAC6D620C3E8A90085D37D
:1019B80060A6D6D00686D36868D0A5CA86D6208702
:1019C800E5A4D584D3604885D78A489848A9008576
:1019D800D0A4D3A5D710034C00E8C90DD0034CD828
:1019E800E8C9209010C960900429DFD002293F205F
:1019F800B8E64CC7E6A6D8F0034CCBE6C914D02EFF
:101A080098D006202DE74C9FE720E8E88884D3206B
:101A1800B2EAC8B1D18891D1C8B1F38891F3C8C4EA
:101A2800D5D0EFA92091D1AD860291F3104DA6D45F
:101A3800F0034CCBE6C912D00285C7C913D00320E6
:101A480081E5C91DD017C820FAE884D388C4D59089
:101A580009C6D620C3E8A00084D34CDCE6C911D05F
:101A68001D18986916A8E6D6C5D590ECF0EAC6D632
:101A7800E916900485D3D0F820C3E84CDCE62012A0
:101A8800E94C21EDEAEAEAEAEAEAEAEAEAEAEAEA13
:101A9800EAEAEAEAEAEAEAEAEA297FC97FD002A999
:101AA8005EEAEAEAEAEAEAC92090034CC5E6C90D0B
:101AB800D0034CD8E8A6D4D03FC914D037A4D5B1A8
:101AC800D1C920D004C4D3D007C057F02420EEE9F0
:101AD800A4D520B2EA88B1D1C891D188B1F3C89110
:101AE800F388C4D3D0EFA92091D1AD860291F3E653
:101AF800D84CDCE6A6D8F00509404CCBE6C911D095
:101B080016A6D6F037C6D6A5D338E916900485D3DD
:101B1800102A2087E5D025C912D004A90085C7C995
:101B28001DD01298F00920E8E88884D34CDCE62020
:101B38002DE74CDCE6C913D006205FE54CDCE6094E
:101B4800802012E94C30ED46C9A6D6E8E017D0034C
:101B58002075E9B5D910F486D64C87E5A20086D859
:101B680086C786D486D320C3E84CDCE6A204A90045
:101B7800C5D3F007186916CAD0F660C6D660A204A5
:101B8800A915C5D3F007186916CAD0F660A6D6E01D
:101B980017F002E6D660A207DD21E9F004CA10F8C2
:101BA800608E86026090051C9F9C1E1F9EEFA1DF21
:101BB800A6E1B1E2B2E3B3E4B4E5B5E6B6E7B7E867
:101BC800B8E9B9FABAFBBBFCBCECBDFEBE84BFF7F2
:101BD800C0F8DBF9DDEADE5EE05BE15DE240B061C2
:101BE800B178DB79DD66B677C070F071F172F273A7
:101BF800F374F475F576F67DFDA5AC48A5AD48A55A
:101C0800AE48A5AF48A2FFC6D6C6C9C6F2E8207E30
:101C1800EAE016B00CBDFEED85ACB5DA2056EA3028
:101C2800EC208DEAA200B5D9297FB4DA1002098028
:101C380095D9E8E016D0EFA5EF098085EFA5D91072
:101C4800C4E6D6E6F2A9FB8D2091AD2191C9FE0824
:101C5800A9F78D209128D00BA000EACAD0FC88D023
:101C6800F984C6A6D66885AF6885AE6885AD6885EF
:101C7800AC60A6D6E8B5D910FB86F2E016F00D9058
:101C88000B2075E9A6F2CAC6D64C0EE7A5AC48A546
:101C9800AD48A5AE48A5AF48A217CA207EEAE4F22F
:101CA800900EF00CBDFCED85ACB5D82056EA30EAB4
:101CB800208DEAA215E4F2900FB5DA297FB4D91085
:101CC80002098095DACAD0EDA6F2200EE76885AF42
:101CD8006885AE6885AD6885AC6029030D88028586
:101CE800AD206EEAA015B1AC91D1B1AE91F38810D8
:101CF800F56020B2EAA5AC85AEA5AD2903099485A7
:101D0800AF60BDFDED85D1B5D929030D880285D217
:101D180060A015207EEA20B2EAA92091D1A90191FC
:101D2800F38810F560A8A90285CD20B2EA98A4D35B
:101D380091D18A91F360A5D185F3A5D2290309949D
:101D480085F46020EAFFA5CCD029C6CDD025A914FA
:101D580085CDA4D346CFAE8702B1D1B011E6CF85E9
:101D6800CE20B2EAB1F38D8702AE8602A5CE4980B5
:101D780020AAEAAD1F912940F00BA00084C0AD1C39
:101D8800910902D009A5C0D00DAD1C9129FD2C1ECA
:101D98009170038D1C91201EEB2C249168A868AAD1
:101DA8006840A9008D8D02A04084CB8D2091AE2182
:101DB80091E0FFF05EA9FE8D2091A000A95E85F557
:101DC800A9EC85F6A208AD2191CD2191D0F64AB0B3
:101DD8001648B1F5C905B00CC903F0080D8D028D80
:101DE8008D02100284CB68C8C041B009CAD0DF3860
:101DF8002E2091D0CF6C8F02A4CBB1F5AAC4C5F028
:101E080007A0108C8C02D036297F2C8A02301670DD
:101E180049C97FF029C914F00CC920F008C91DF080
:101E280004C911D035AC8C02F005CE8C02D02BCE73
:101E38008B02D026A0048C8B02A4C688101CA4CBCD
:101E480084C5AC8D028C8E02E0FFF00E8AA6C6EC2B
:101E58008902B0069D7702E886C6A9F78D209160B1
:101E6800AD8D02C903D02CCD8E02F0EEAD910230BB
:101E780056EAEAEAEAEAEAEAEAEAEAEAEAEAEAEA4E
:101E8800EAEAEAEAAD059049028D0590EAEAEAEA4B
:101E98004C43EC0AC9089004A906EAEAEAEAEAEA25
:101EA800EAEAEAEAEAEAEAEAEAEAEAEAEAEAEAEA8A
:101EB800EAEAEAEAEAEAEAEAEAEAEAEAAABD46EC89
:101EC80085F5BD47EC85F64C74EB5EEC9FECE0ECD9
:101ED800A3ED5EEC9FEC69EDA3ED21ED69ED69EDF5
:101EE800A3ED31333537392B5C145F5752594950BC
:101EF8002A0D044144474A4C3B1D030158564E2CB9
:101F08002F11205A43424D2E0185025346484B3A21
:101F18003D86514554554F405E8732343638302D12
:101F28001388FF2123252729DBA9945FD7D2D9C994
:101F3800D0C08D04C1C4C7CACC5D9D8301D8D6CE9C
:101F48003C3F91A0DAC3C2CD3E018902D3C6C8CBBB
:101F58005B3D8AD1C5D4D5CFBADE8B222426283062
:101F6800DD938CFF2123252729A6A8945FB3B2B758
:101F7800A2AFDF8D04B0ACA5B5B65D9D8301BDBE33
:101F8800AA3C3F91A0ADBCBFA73E018902AEBBB43D
:101F9800A15B3D8AABB1A3B8B9A4DE8B2224262865
:101FA80030DC938CFFC90ED00BA9020D05908D056E
:101FB800904CDCE6C98ED00BA9FD2D05908D0590BF
:101FC8004CDCE6C908D00AA9800D91028D91023037
:101FD800EFC909D0EBA97F2D91028D910210E1E89C
:101FE800B5D9098095D9CAA5D5184C15E7FFFFFFC3
:101FF800FFFFFFFFFFFF04FFFFFFFFFFE29D8301DD
:10200800FFFFFFFFFF91A0FFFFFFFFEE018902FF27
:10201800FFFFFFE1FD8AFFFFFFFFFFB0E08BF2F457
:10202800F6FFF0ED938CFF901C9C1F12FFFFFF063C
:10203800FF12FFFFFFFFFFFFFFFFFFFFFFFFFFFF95
:10204800FFFFFFFFFFFFFFFFFFFFFFFFFFFFFFFF98
:10205800FFFFFFFFFFFFFFFFFFFFFFFFFFFFFF0582
:102068009F1E9E92FFFFFFFF0519162E00C000005D
:10207800000000000000001B4C4F41440D52554E1B
:102088000D00162C42586E849AB0C6DCF2081E3435
:102098004A60768CA2B8CEE409402C09202060F171
:1020A800482494100A3866A32049EE469446A3684B
:1020B800859520A0E4C93FD0032084EFAD1F910986
:1020C800808D1F91208DEF20A0E42096EF7820A02E
:1020D800E420B2E44AB0612084EF24A3100C20B2BB
:1020E800E44A90FA20B2E44AB0FA20B2E44A90FAFC
:1020F800208DEFA90885A5AD1F91CD1F91D0F84A75
:102108004A90386695B00520A9E4D00320A0E420C1
:1021180084EFEAEAEAEAAD2C9129DF09028D2C91D5
:10212800C6A5D0D3A9048D2991AD2D912920D00B16
:1021380020B2E44AB0F35860A9802CA903206AFEB3
:102148005818904985952040EEAD1F91297F8D1F25
:10215800916085952040EE7820A9E420C5EE208482
:10216800EF20B2E4B0FB586024943005386694D070
:1021780005482049EE6885951860208DEFAD1F91C0
:1021880009808D1F91A95F2CA93F201CEE20C5EE68
:102198008AA20BCAD0FDAA2084EF4CA0E478A9003B
:1021A80085A52084EF20B2E490FB20A0E4A9018D4E
:1021B8002991AD2D912920D00720B2E4B0F49018D0
:1021C800A5A5F005A9024CB9EE20A9E4200CEFA9B9
:1021D80040206AFEE6A5D0D5A90885A5AD1F91CDFA
:1021E8001F91D0F84A90F54A66A4AD1F91CD1F9172
:1021F800D0F84AB0F5C6A5D0E320A9E4A590F0032D
:10220800200CEFA5A4581860AD2C9129FD8D2C91B8
:1022180060AD2C9109028D2C9160A9048D2991AD96
:102228002D912920F0F960A5B4F047303F46B6A2B9
:10223800009001CA8A45BD85BDC6B4F0068A29202A
:1022480085B560A9202C9402F014301C7014A5BD2B
:10225800D001CAC6B4AD930210E3C6B4D0DFE6B469
:10226800D0F0A5BDF0EDD0EA70E950E6E6B4A2FFE3
:10227800D0CBAD94024A90072C2091101D501EA976
:102288000085BD85B5AE980286B4AC9D02CC9E0291
:10229800F013B1F985B6EE9D0260A9402CA9100D86
:1022A80097028D9702A9408D1E9160A209A9202C42
:1022B8009302F001CA5002CACA60A6A9D02EC6A8C5
:1022C800F031300DA5A745AB85AB46A766AA60C619
:1022D800A8A5A7F062AD93020AA90165A8D0EFA945
:1022E800908D1E9185A9A9208D1E9160A5A7D0EF7C
:1022F80085A960AC9B02C8CC9C02F02A8C9B028802
:10230800A5AAAE9802E009F0044AE8D0F891F7A926
:10231800202C9402F0B930B6A5A745ABF00370AEF7
:102328002C50ABA9012CA9042CA9802CA9020D972B
:10233800028D97024C5BF0A5AAD0F1F0EC4C96F711
:10234800859AAD94024A9027A9022C1091101DD0AD
:102358001EAD1E912930D0F92C109170FBAD109153
:1023680009028D10912C1091700530F92016F01883
:1023780060AC9E02C8CC9D02F0F78C9E028891F951
:102388002C1E91500160AD99028D1491AD9A028D69
:102398001591A9C08D1E914CEEEF8599AD94024A16
:1023A80090282908F024A9022C109110BFF0192CAC
:1023B8001E9170FBAD109129FD8D1091AD109129E2
:1023C80004F0F9A9908D1E911860AD1E912930F086
:1023D800F21860AC9C02CC9B02F006B1F7EE9C02AE
:1023E80060A9006048AD1E91F00CAD1E912960D027
:1023F800F9A9108D1E9168600D492F4F2045525242
:102408004F5220A30D534541524348494E47A046D9
:102418004F52A00D505245535320504C4159204F14
:102428004E20544150C55052455353205245434FB6
:102438005244202620504C4159204F4E20544150A0
:10244800C50D4C4F4144494EC70D534156494E475F
:10245800A00D564552494659494EC70D464F554E4F
:1024680044A00D4F4B8D249D100DB974F108297FA0
:1024780020D2FFC82810F31860A599D008A5C6F087
:102488006D784CCFE5C902D0188497204FF1A497F6
:102498001860A599D00BA5D385CAA5D685C94C4F78
:1024A800E6C903D00985D0A5D585C84C4FE6B03814
:1024B800C902F03F86972050F2B016482050F2B07B
:1024C8000DD005A940206AFEC6A6A6976860AA682E
:1024D8008AA69760208AF8D00B20C0F8B011A9000E
:1024E80085A6F0F0B1B21860A590F004A90D1860A7
:1024F8004C19EF2005F2B005C900F0F7186048A59F
:102508009AC903D004684C42E79004684CE4EEC9C9
:1025180002F02A68859E488A489848208AF8D00E92
:1025280020E3F8B00EA902A00091B2C884A6A59E27
:1025380091B21868A868AA689002A900606886978E
:10254800849E20EDF0A697A49E186020CFF3F00398
:102558004C84F720DFF3A5BAF016C903F012B014C3
:10256800C902D0034C16F1A6B9E060F0034C8DF710
:1025780085991860AA2014EEA5B9100620D3EE4C50
:1025880001F320CEEE8A249010E64C8AF720CFF390
:10259800F0034C84F720DFF3A5BAD0034C90F7C9B9
:1025A80003F00FB011C902D0034CBCF0A6B9E0602B
:1025B800F0EA859A1860AA2017EEA5B9100520C57B
:1025C800EED00320C0EE8A249010E74C8AF720D47E
:1025D800F3F002186020DFF38A48A5BAF057C90360
:1025E800F053B04EC902D0296820B2F3A97D8D1EE0
:1025F80091A9068D1091A9EE8D1C912075FEA5F864
:10260800F001C8A5FAF001C8A90085F885FA4C3C84
:10261800F5A5B9290FF01E204DF8A9002090F24C1D
:10262800CFE4B02EA5B9C962D00BA90520E7F74CB5
:10263800B1F320DAF668AAC698E498F014A498B919
:1026480059029D5902B963029D6302B96D029D6DDD
:10265800021860A90085908AA698CA3015DD59022B
:10266800D0F860BD590285B8BD630285BABD6D0258
:1026780085B960A9008598A203E49AB0032004EF05
:10268800E499B00320F6EE869AA900859960A6B869
:10269800D0034C8DF720CFF3D0034C81F7A698E0F8
:1026A8000A90034C7EF7E698A5B89D5902A5B9098A
:1026B8006085B99D6D02A5BA9D6302F05AC903F001
:1026C8005690052095F4904FC902D0034CC7F420CA
:1026D8004DF8B0034C96F7A5B9290FD01F2094F8F0
:1026E800B0362047F6A5B7F00A2067F89018F0280A
:1026F8004C87F720AFF7F020900CB0F420B7F8B073
:1027080017A90420E7F7A9BFA4B9C060F007A00083
:10271800A90291B29885A61860A5B9302CA4B7F083
:1027280028A5BA2017EEA5B909F020C0EEA590108B
:102738000568684C8AF7A5B7F00CA000B1BB20E487
:10274800EEC8C4B7D0F62004EF1860A9068D129120
:102758008D1091A9EE8D1C91A0008C9702C4B7F042
:102768000AB1BB999302C8C004D0F22027F08E9812
:1027780002AD9302290FD0000AAABD5AFF0AA8BDCC
:102788005BFF2A489869C88D99026869008D9A028A
:10279800AD94024A9009AD20910AB0034C16F0ADF1
:1027A8009B028D9C02AD9E028D9D022075FEA5F8B0
:1027B800D0058884F886F7A5FAD0058884FA86F9C2
:1027C80038A9F04C7BFE86C384C46C30038593A97A
:1027D800008590A5BAD0034C96F7C903F0F9906E1E
:1027E800A4B7D0034C93F720BCE4A96085B9209521
:1027F800F4A5BA2014EEA5B920CEEE2019EF85AEC7
:10280800A5904A4AB0452019EF85AF20C1E4A9FD3B
:102818002590859020E1FFD0034CCBF62019EFAA34
:10282800A5904A4AB0E88AA493F00CA000D1AEF073
:1028380008A910206AFE2C91AEE6AED002E6AF24BD
:102848009050CB20F6EE20DAF6907A4C87F7C90242
:10285800D0034CB9F0204DF8B0034C96F72094F80B
:10286800B0682047F6A5B7F0092067F8900BF05A32
:10287800B0D920AFF7F053B0D2A590291038D04A7C
:10288800E001F011E003D0DDA001B1B285C3C8B109
:10289800B285C4B004A5B9D0EFA003B1B2A001F1CC
:1028A800B2AAA004B1B2A002F1B2A8188A65C38581
:1028B800AE9865C485AFA5C385C1A5C485C2206A85
:1028C800F620C9F82418A6AEA4AF60A59D101EA0D6
:1028D8000C20E6F1A5B7F015A01720E6F1A4B7F093
:1028E8000CA000B1BB20D2FFC8C4B7D0F660A04985
:1028F800A593F002A0594CE2F186AE84AFAAB500C8
:1029080085C1B50185C26C3203A5BAD0034C96F7D0
:10291800C903F0F9905FA96185B9A4B7D0034C93B6
:10292800F72095F42028F7A5BA2017EEA5B920C0FE
:10293800EEA00020D2FBA5AC20E4EEA5AD20E4EE8D
:102948002011FDB016B1AC20E4EE20E1FFD0072045
:10295800DAF6A9003860201BFDD0E52004EF24B981
:102968003011A5BA2017EEA5B929EF09E020C0EE6D
:102978002004EF1860C902D0034CB9F0204DF8903C
:102988008C20B7F8B0252028F7A203A5B92901D0D3
:1029980002A2018A20E7F7B01220E6F8B00DA5B927
:1029A8002902F006A90520E7F7241860A59D10FB69
:1029B800A05120E6F14C59F6A200E6A2D006E6A105
:1029C800D002E6A038A5A2E901A5A1E91AA5A0E9C7
:1029D8004F900686A086A186A2AD2F91CD2F91D0CB
:1029E800F885916078A5A2A6A1A4A07885A286A161
:1029F80084A05860A591C9FED0070820CCFF85C6E1
:102A08002860A9012CA9022CA9032CA9042CA9052A
:102A18002CA9062CA9072CA9082CA9094820CCFF09
:102A2800A000249D500A20E6F16848093020D2FF12
:102A3800683860A5934820C0F8688593B02CA0003A
:102A4800B1B2C905F024C901F008C903F004C904EA
:102A5800D0E1AA249D1011A06320E6F1A005B1B22F
:102A680020D2FFC8C015D0F6188860859E204DF882
:102A7800905EA5C248A5C148A5AF48A5AE48A0BF6D
:102A8800A92091B288D0FBA59E91B2C8A5C191B2E8
:102A9800C8A5C291B2C8A5AE91B2C8A5AF91B2C837
:102AA800849FA000849EA49EC4B7F00CB1BBA49FD1
:102AB80091B2E69EE69FD0EE2054F8A96985AB2036
:102AC800EAF8A86885AE6885AF6885C16885C29848
:102AD80060A6B2A4B3C00260204DF88A85C1186907
:102AE800C085AE9885C2690085AF6020AFF7B01D7C
:102AF800A005849FA000849EC4B7F010B1BBA49F1A
:102B0800D1B2D0E7E69EE69FA49ED0EC1860204D97
:102B1800F8E6A6A4A6C0C06020ABF8F01CA01B2055
:102B2800E6F1204BF920ABF8D0F8A06A4CE6F1A901
:102B3800402C1F91D0032C1F91186020ABF8F0F99E
:102B4800A02ED0DBA900859085932054F82094F816
:102B5800B01F78A90085AA85B485B0859E859F8514
:102B68009CA982A20ED0112054F8A91485AB20B7D5
:102B7800F8B06878A9A0A208A07F8C2E918D2E911C
:102B88002060F1AD14038D9F02AD15038DA00220C6
:102B9800FBFCA90285BE20DBFBAD1C9129FD090CBD
:102BA8008D1C9185C0A2FFA0FF88D0FDCAD0F88DEA
:102BB800299158ADA002CD150318F01F204BF9AD8F
:102BC8002D912940F0EDAD14912034F74C2FF920C8
:102BD800E1FF18D00B20CFFC386868A9008DA0024F
:102BE8006086B1A5B00A0A1865B01865B185B1A9A3
:102BF8000024B030012A06B12A06B12AAAAD2891CC
:102C0800C91590F965B18D24918A6D29918D259109
:102C18005860AE2991A0FF98ED2891EC2991D0F247
:102C280086B1AA8C28918C299198E5B186B14A661B
:102C3800B14A66B1A5B018693C2C2191C5B1B04A1A
:102C4800A69CF0034CADFAA6A3301BA20069306520
:102C5800B0C5B1B01CE8692665B0C5B1B017692C1C
:102C680065B0C5B190034C60FAA5B4F01D85A8D035
:102C780019E6A9B002C6A938E913E5B165928592AB
:102C8800A5A4490185A4F02186D7A5B4F0182C2D58
:102C9800915013A90085A4A5A3103030C9A2A6207D
:102CA8005DF9A59BD0C34C56FFA592F0073003C62B
:102CB800B02CE6B0A9008592E4D7D00F8AD0AAA597
:102CC800A930C7C91090C38596B0BF8A459B859B1C
:102CD800A5B4F0D2C6A330C546D766BFA2DA205D38
:102CE800F94C56FFA596F004A5B4F004A5A31085E9
:102CF80046B1A99338E5B165B00AAA205DF9E69C0A
:102D0800A5B4D011A596F02685A8A9008596A9C0D6
:102D18008D2E9185B4A59685B5F009A90085B4A92D
:102D2800408D2E91A5BF85BDA5A805A985B64C5691
:102D3800FF20DBFB859CA2DA205DF9A5BEF00285A9
:102D4800A7A90F24AA1017A5B5D00CA6BECAD00BE8
:102D5800A908206AFED004A90085AA4C56FF703144
:102D6800D018A5B5D0F5A5B6D0F1A5A74AA5BD3010
:102D780003901818B015290F85AAC6AAD0DDA94056
:102D880085AA20D2FBA90085ABF0D0A98085AAD05E
:102D9800CAA5B5F00AA904206AFEA9004C97FB2031
:102DA80011FD90034C95FBA6A7CAF02DA593F00C36
:102DB800A000A5BDD1ACF004A90185B6A5B6F04B1D
:102DC800A23DE49E903EA69EA5AD9D0101A5AC9DA9
:102DD8000001E8E8869E4C87FBA69FE49EF035A597
:102DE800ACDD0001D02EA5ADDD0101D027E69FE6C0
:102DF8009FA593F00BA5BDA000D1ACF017C884B671
:102E0800A5B6F007A910206AFED009A593D005A899
:102E1800A5BD91AC201BFDD03AA98085AAA6BECA43
:102E2800300286BEC6A7F008A59ED02785BEF0232F
:102E380020CFFC20D2FBA00084ABB1AC45AB85AB66
:102E4800201BFD2011FD90F2A5AB45BDF005A92082
:102E5800206AFE4C56FFA5C285ADA5C185AC60A908
:102E68000885A3A90085A485A8859B85A960A5BD1B
:102E78004AA9609002A9B0A2008D28918E2991AD2F
:102E8800209149088D20912908603866AD303CA50D
:102E9800A8D012A910A20120F5FBD02FE6A8A5AD55
:102EA80010294C95FCA5A9D00920F1FBD01DE6A955
:102EB800D01920EAFBD014A5A4490185A4F00FA5D8
:102EC800BD490185BD2901459B859B4C56FF46BDE3
:102ED800C6A3A5A3F03A10F320DBFB58A5A5F01272
:102EE800A20086D7C6A5A6BEE002D002098085BD8D
:102EF800D0D92011FD900AD091E6ADA5D785BDB0F7
:102F0800CAA000B1AC85BD45D785D7201BFDD0BB75
:102F1800A59B490185BD4C56FFC6BED0032008FDC0
:102F2800A95085A7A2087820FBFCD0EAA97820F34D
:102F3800FBD0E3C6A7D0DF20DBFBC6AB10D8A20AC4
:102F480020FBFC58E6ABA5BEF03020D2FBA20986D8
:102F5800A5D08508782008FDA97F8D2E91A9F78D29
:102F68002091A9408D2B912039FEADA002F0098D4A
:102F78001503AD9F028D1403286020CFFCF097BD88
:102F8800E9FD8D1403BDEAFD8D150360AD1C9109A3
:102F98000E8D1C916038A5ACE5AEA5ADE5AF60E639
:102FA800ACD002E6AD60A2FF789AD8203FFDD003EE
:102FB8006C00A0208DFD2052FD20F9FD2018E55859
:102FC8006C00C0A205BD4CFDDD03A0D003CAD0F53E
:102FD800604130C3C2CDA26DA0FD1886C384C4A0D1
:102FE8001FB91403B002B1C391C39914038810F137
:102FF80060BFEAD2FEADFE0AF44AF3C7F209F3F362
:10300800F30EF27AF270F7F5F1EFF3D2FE49F58597
:10301800F6A900AA95009D00029D0003E8D0F5A23C
:103028003CA00386B284B385C185978D8102A8A987
:103038000485C2E6C1D002E6C22091FEA597F0221F
:10304800B0F1A4C2A6C1C0209025C021B008A01E1E
:103058008C88024C7BFEA9128D8202A9108D8802F1
:10306800D0F190CFA5C28D82028597C91190C42056
:10307800C3E54CEBFDA8FC0BFCBFEA8EF9A97F8DDC
:103088001E918D2E91A9408D2B91A9408D1B91A940
:10309800FE8D1C91A9DE8D2C91A2008E1291A2FFAB
:1030A8008E2291A2008E2391A2808E1391A2008E6F
:1030B8001F912084EFA9828D1E91208DEFA9C08DCC
:1030C8002E91A9898D2491A9428D25916085B78675
:1030D800BB84BC6085B886BA84B960A5BAC902D079
:1030E8000BAD9702A9008D970260859DA59005906C
:1030F8008590608D8502609006AE8302AC84028E56
:1031080083028C8402609006AE8102AC82028E81BA
:10311800028C820260B1C1AAA95591C1D1C1D0085F
:103128006A91C1D1C1D001A9188A91C160786C187F
:1031380003488A489848AD1D9110482D1E91AA2928
:1031480002F01F203FFDD0036C02A02C1191203407
:10315800F720E1FFD02D2052FD20F9FD2018E56C65
:1031680002C0AD1E91098048A97F8D1E918A294011
:10317800F014A9CE05B58D1C91AD1491688D1E91E2
:1031880020A3EF4C56FF8A2920F025AD1091290184
:1031980085A7AD1891E9166D99028D1891AD199111
:1031A8006D9A028D1991688D1E912036F04C56FF4C
:1031B8008A2910F025AD9302290FD0000AAABD5A1A
:1031C800FF8D1891BD5BFF8D1991AD109168092095
:1031D80029EF8D1E91AE980286A868A868AA684053
:1031E8009227401AC611740EEE0C4506F1024601EC
:1031F800B80071002A00488A489848BABD040129D5
:1032080010F0036C16036C1403FFFFFFFFFF4C5212
:10321800FD4C57FD4C66FE4CC0EE4CCEEE4C73FE9A
:103228004C82FE4C1EEB4C6FFE4C19EF4CE4EE4CFE
:10323800F6EE4C04EF4C17EE4C14EE4C57FE4C5087
:10324800FE4C49FE6C1A036C1C036C1E036C2003B5
:103258006C22036C24036C26034C42F54C75F64C27
:1032680067F74C60F76C28036C2A036C2C034C340A
:10327800F74C05E54C0AE54C00E5FFFFFFFFA9FE0A
:1032880022FD72FF78E367E443424D4241534943CC
:1032980030C841C71DCDF7C8A4CBBECB80D005CC64
:1032A800A4C99FC870C827C91CC882C8D1C83AC950
:1032B8002EC84AC92CD864E152E161E1B2D323D8BF
:1032C8007FCA9FCA56C89BC65DC685CA26E1BAE1B1
:1032D800C3E17ACB41C639DCCCDC58DC00007DD3B5
:1032E8009ED371DF94E0EAD9EDDF61E268E2B1E2F2
:1032F8000BE30DD87CD765D4ADD78BD7ECD600D7E8
:103308002CD737D77969D87952D87B2ADA7B11DB61
:103318007F7ADF50E8CF46E5CF7DB3DF5AD3CE645E
:1033280015D0454EC4464FD24E4558D4444154C199
:10333800494E505554A3494E5055D44449CD524551
:1033480041C44C45D4474F54CF5255CE49C6524537
:1033580053544F52C5474F5355C25245545552CEF8
:103368005245CD53544FD04FCE574149D44C4F417D
:10337800C4534156C55645524946D94445C6504F8F
:103388004BC55052494E54A35052494ED4434F4E08
:10339800D44C4953D4434CD2434DC45359D34F50C2
:1033A80045CE434C4F53C54745D44E45D75441426B
:1033B800A854CF46CE535043A8544845CE4E4FD478
:1033C800535445D0ABADAAAFDE414EC44FD2BEBDBB
:1033D800BC5347CE494ED44142D35553D24652C529
:1033E800504FD35351D2524EC44C4FC74558D04377
:1033F8004FD35349CE5441CE4154CE504545CB4C82
:1034080045CE535452A45641CC4153C3434852A4C9
:103418004C454654A45249474854A44D4944A447EE
:10342800CF00544F4F204D414E592046494C45D36B
:1034380046494C45204F5045CE46494C45204E4FB5
:1034480054204F5045CE46494C45204E4F542046B7
:103458004F554EC4444556494345204E4F5420507D
:10346800524553454ED44E4F5420494E5055542042
:1034780046494CC54E4F54204F555450555420463C
:10348800494CC54D495353494E472046494C452060
:103498004E414DC5494C4C4547414C204445564941
:1034A8004345204E554D4245D24E45585420574924
:1034B80054484F555420464FD253594E5441D85230
:1034C800455455524E20574954484F555420474F5C
:1034D8005355C24F5554204F4620444154C1494C7E
:1034E8004C4547414C205155414E544954D94F56AB
:1034F8004552464C4FD74F5554204F46204D454DC9
:103508004F52D9554E4445462744205354415445BB
:103518004D454ED44241442053554253435249509D
:10352800D4524544494D27442041525241D9444937
:10353800564953494F4E204259205A4552CF494C7B
:103548004C4547414C204449524543D45459504571
:10355800204D49534D415443C8535452494E472076
:10356800544F4F204C4F4EC746494C452044415478
:10357800C1464F524D554C4120544F4F20434F4D5B
:10358800504C45D843414E275420434F4E54494E42
:1035980055C5554E44454627442046554E43544943
:1035A8004FCE5645524946D94C4F41C49EC1ACC135
:1035B800B5C1C2C1D0C1E2C1F0C1FFC110C225C2AC
:1035C80035C23BC24FC25AC26AC272C27FC290C2DF
:1035D8009DC2AAC2BAC2C8C2D5C2E4C2EDC200C363
:1035E8000EC31EC324C383C30D4F4B0D000D2045CE
:1035F80052524F520020494E20000D0A5245414474
:10360800592E0D0A000D0A425245414B00A0BAE856
:10361800E8E8E8BD0101C981D021A54AD00ABD0268
:10362800018549BD0301854ADD0301D007A549DDB0
:103638000201F0078A186912AAD0D8602008C48548
:1036480031843238A55AE55F8522A8A55BE560AAD2
:10365800E898F023A55A38E522855AB003C65B38A6
:10366800A558E5228558B008C6599004B15A915812
:1036780088D0F9B15A9158C65BC659CAD0F2600AC7
:10368800693EB0358522BAE422902E60C434902871
:10369800D004C533902248A2099848B557CA10FAF1
:1036A8002026D5A2F7689561E830FA68A868C4347E
:1036B8009006D005C533B00160A2106C00038A0AD9
:1036C800AABD26C38522BD27C3852320CCFFA90018
:1036D800851320D7CA2045CBA000B12248297F20D6
:1036E80047CBC86810F4207AC6A969A0C3201ECBAE
:1036F800A43AC8F00320C2DDA976A0C3201ECBA936
:10370800802090FF6C02032060C5867A847B20733A
:1037180000AAF0F0A2FF863A90062079C54CE1C7CE
:10372800206BC92079C5840B2013C69044A001B131
:103738005F8523A52D8522A5608525A55F88F15F76
:1037480018652D852D8524A52E69FF852EE560AA8F
:1037580038A55FE52DA8B003E8C6251865229003B3
:10376800C62318B1229124C8D0F9E623E625CAD089
:10377800F22059C62033C5AD0002F08818A52D8562
:103788005A650B8558A42E845B9001C8845920B8CB
:10379800C3A514A4158DFE018CFF01A531A43285A3
:1037A8002D842EA40B88B9FC01915F8810F820594C
:1037B800C62033C54C80C4A52BA42C85228423188D
:1037C800A001B122F01DA004C8B122D0FBC89865A1
:1037D80022AAA0009122A5236900C89122862285E9
:1037E8002390DD60A200200FE1C90DF00D9D0002BD
:1037F800E8E05990F1A2174C37C44CCACA6C0403CC
:10380800A67AA004840FBD00021007C9FFF03EE8A5
:10381800D0F4C920F0378508C922F056240F702D3E
:10382800C93FD004A999D025C9309004C93C901D3E
:103838008471A000840B88867ACAC8E8BD00023863
:10384800F99EC0F0F5C980D030050BA471E8C8997D
:10385800FB01B9FB01F03638E93AF004C949D00256
:10386800850F38E955D09F8508BD0002F0DFC508EF
:10387800F0DBC899FB01E8D0F0A67AE60BC8B99D41
:10388800C010FAB99EC0D0B4BD000210BE99FD01A7
:10389800C67BA9FF857A60A52BA62CA001855F862B
:1038A80060B15FF01FC8C8A515D15F9018F00388F4
:1038B800D009A51488D15F900CF00A88B15FAA8856
:1038C800B15FB0D71860D0FDA900A8912BC8912B83
:1038D800A52B186902852DA52C6900852E208EC67A
:1038E800A900D02D20E7FFA537A43885338434A557
:1038F8002DA42E852F843085318432201DC8A2192D
:10390800861668A868A2FA9A489848A900853E854C
:10391800106018A52B69FF857AA52C69FF857B6047
:103928009006F004C9ABD0E9206BC92013C62079F2
:1039380000F00CC9ABD08E207300206BC9D086680C
:1039480068A5140515D006A9FF85148515A001845E
:103958000FB15FF043202CC820D7CAC8B15FAAC8EE
:10396800B15FC515D004E414F002B02C844920CD11
:10397800DDA920A449297F2047CBC922D006A50F5D
:1039880049FF850FC8F011B15FD010A8B15FAAC870
:10399800B15F865F8560D0B54C74C46C060310D7E0
:1039A800C9FFF0D3240F30CF38E97FAA8449A0FF9C
:1039B800CAF008C8B99EC010FA30F5C8B99EC03020
:1039C800B22047CBD0F5A980851020A5C9208AC38D
:1039D800D0058A690FAA9A6868A90920FBC320063E
:1039E800C91898657A48A57B690048A53A48A53959
:1039F80048A9A420FFCE208DCD208ACDA566097FB9
:103A080025628562A98BA0C7852284234C43CEA951
:103A1800BCA0D920A2DB207900C9A9D00620730058
:103A2800208ACD202BDC2038CEA54A48A54948A9B4
:103A38008148202CC8A57AA47BC002EAF004853D01
:103A4800843EA000B17AD043A002B17A18D0034CCA
:103A58004BC8C8B17A8539C8B17A853A98657A85EC
:103A68007A9002E67B6C080320730020EDC74CAE09
:103A7800C7F03CE9809011C923B0170AA8B90DC056
:103A880048B90CC0484C73004CA5C9C93AF0D64C8B
:103A980008CFC94BD0F9207300A9A420FFCE4CA0B1
:103AA800C838A52BE901A42CB0018885418442605F
:103AB80020E1FFB00118D03CA57AA47BA63AE8F033
:103AC8000C853D843EA539A43A853B843C6868A9A9
:103AD80081A0C390034C69C44C74C4D017A21AA423
:103AE8003ED0034C37C4A53D857A847BA53BA43CD6
:103AF8008539843A6008A9002090FF28D0034C59E2
:103B0800C62060C64C97C8A90320FBC3A57B48A55F
:103B18007A48A53A48A53948A98D4820790020A0B7
:103B2800C84CAEC7206BC92009C938A539E514A50A
:103B38003AE515B00B9838657AA67B9007E8B0048B
:103B4800A52BA62C2017C6901EA55FE901857AA58E
:103B580060E900857B60D0FDA9FF854A208AC39A69
:103B6800C98DF00BA20C2CA2114C37C44C08CF689D
:103B780068853968853A68857A68857B2006C9989A
:103B880018657A857A9002E67B60A23A2CA20086B4
:103B980007A0008408A508A60785078608B17AF05B
:103BA800E8C508F0E4C8C922D0F3F0E9209ECD208A
:103BB8007900C989F005A9A720FFCEA561D0052005
:103BC80009C9F0BB207900B0034CA0C84CEDC72050
:103BD8009ED748C98DF004C989D091C665D00468BC
:103BE8004CEFC7207300206BC9C92CF0EE6860A2A7
:103BF8000086148615B0F7E92F8507A5158522C913
:103C080019B0D4A5140A26220A262265148514A5FB
:103C1800226515851506142615A5146507851490C3
:103C280002E6152073004C71C9208BD08549844A5F
:103C3800A9B220FFCEA50E48A50D48209ECD682A22
:103C48002090CDD018681012201BDC20BFD1A00016
:103C5800A5649149C8A5659149604CD0DB68A44A20
:103C6800C0DFD04C20A6D6C906D03DA00084618410
:103C7800668471201DCA20E2DAE671A471201DCA8B
:103C8800200CDCAAF005E88A20EDDAA471C8C00689
:103C9800D0DF20E2DA209BDCA664A463A5654CDBB8
:103CA800FFB12220800090034C48D2E92F4C7EDDE2
:103CB800A002B164C5349017D00788B164C53390A9
:103CC8000EA465C42E9008D00DA564C52DB007A517
:103CD80064A4654C68CAA000B1642075D4A550A43A
:103CE80051856F8470207AD6A961A00085508451CF
:103CF80020DBD6A000B1509149C8B1509149C8B154
:103D0800509149602086CA4CB5CB209ED7F005A9B2
:103D18002C20FFCE0886132015E1284CA0CA2021AC
:103D2800CB207900F035F043C9A3F050C9A618F0AC
:103D38004BC92CF037C93BF05E209ECD240D30DEF8
:103D480020DDDD2087D42021CB203BCBD0D3A90098
:103D58009D0002A2FFA001A513D010A90D2047CBFA
:103D680024131005A90A2047CB49FF603820F0FF2B
:103D78009838E90BB0FC49FF6901D016083820F0E3
:103D8800FF8409209BD7C929D0592890068AE509BC
:103D98009005AAE8CAD0062073004CA2CA203BCBE3
:103DA800D0F22087D420A6D6AAA000E8CAF0BCB1D9
:103DB800222047CBC8C90DD0F320E5CA4C28CBA593
:103DC80013F003A9202CA91D2CA93F2009E129FFE4
:103DD80060A511F0113004A0FFD004A53FA44085D0
:103DE80039843A4C08CFA513F005A2184C37C4A95A
:103DF8000CA0CD201ECBA53DA43E857A847B6020F7
:103E0800A6D3C923D010207300209ED7A92C20FF49
:103E1800CE8613201BE1A201A002A9008D0102A9F0
:103E280040200FCCA613D01360209ED7A92C20FFCA
:103E3800CE8613201BE120CECBA51320CCFFA200F9
:103E4800861360C922D00B20BDCEA93B20FFCE200F
:103E580021CB20A6D3A92C8DFF0120F9CBA513F0E7
:103E68000D20B7FF2902F00620B5CB4CF8C8AD00ED
:103E780002D01EA513D0E32006C94CFBC8A513D059
:103E8800062045CB203BCB4C60C5A641A442A9984F
:103E98002CA900851186438444208BD08549844A07
:103EA800A57AA47B854B844CA643A444867A847B5C
:103EB800207900D0202411500C2021E18D0002A28D
:103EC800FFA001D00C3075A513D0032045CB20F9F5
:103ED800CB867A847B207300240D1031241150097D
:103EE800E8867AA9008507F00C8507C922F007A99A
:103EF8003A8507A92C188508A57AA47B6900900142
:103F0800C8208DD420E2D720DAC94C91CC20F3DC2C
:103F1800A50E20C2C9207900F007C92CF0034C4D2A
:103F2800CBA57AA47B85438444A54BA44C857A848D
:103F38007B207900F02D20FDCE4C15CC2006C9C879
:103F4800AAD012A20DC8B17AF06CC8B17A853FC860
:103F5800B17AC8854020FBC8207900AAE083D0DC6C
:103F68004C51CCA543A444A61110034C27C8A0006B
:103F7800B143F00BA513D007A9FCA0CC4C1ECB6015
:103F88003F45585452412049474E4F5245440D0031
:103F98003F5245444F2046524F4D205354415254AE
:103FA8000D00D004A000F003208BD08549844A205E
:103FB8008AC3F005A20A4C37C49A8A18690448696A
:103FC80006852468A00120A2DBBABD09018566A583
:103FD80049A44A2067D820D0DBA001205DDCBA388C
:103FE800FD0901F017BD0F018539BD1001853ABDE6
:103FF8001201857ABD1101857B4CAEC78A6911AA69
:104008009A207900C92CD0F12073002024CD209E5D
:10401800CD182438240D3003B00360B0FDA2164C2F
:1040280037C4A67AD002C67BC67AA20024488A483A
:10403800A90120FBC32083CEA900854D2079003833
:10404800E9B19017C903B013C9012A4901454DC503
:104058004D9061854D2073004CBBCDA64DD02CB042
:104068007B69079077650DD0034C3DD669FF8522A3
:104078000A6522A868D980C0B067208DCD48202065
:10408800CE68A44B1017AAF056D05F460D8A2AA610
:104098007AD002C67BC67AA01B854DD0D7D980C0FE
:1040A800B04890D9B982C048B981C0482033CEA55C
:1040B8004D4CA9CD4C08CFA566BE80C0A868852206
:1040C800E6226885239848201BDCA56548A5644836
:1040D800A56348A56248A561486C2200A0FF68F066
:1040E80023C964F003208DCD844B684A8512688506
:1040F8006968856A68856B68856C68856D68856E92
:104108004566856FA561606C0A03A900850D20735B
:1041180000B0034CF3DC2013D190034C28CFC9FF27
:10412800D00FA9A8A0CE20A2DB4C730082490FDAD9
:10413800A1C92EF0DEC9ABF058C9AAF0D1C922D066
:104148000FA57AA47B69009001C82087D44CE2D7D8
:10415800C9A8D013A018D03B20BFD1A56549FFA896
:10416800A56449FF4C91D3C9A5D0034CF4D3C9B475
:1041780090034CA7CF20FACE209ECDA9292CA928A0
:104188002CA92CA000D17AD0034C7300A20B4C3779
:10419800C4A01568684CFACD38A564E900A565E99E
:1041A800C09008A987E564A9E3E56560208BD08500
:1041B800648465A645A446A50DF026A9008570204F
:1041C80014CF901CE054D018C0C9D0142084CF84D8
:1041D8005E888471A006845DA0242068DE4C6FD4BC
:1041E80060240E100DA000B164AAC8B164A88A4C5E
:1041F80091D32014CF902DE054D01BC049D0252056
:1042080084CF98A2A04C4FDC20DEFF8664846385AF
:1042180065A000846260E053D00AC054D00620B77D
:10422800FF4C3CDCA564A4654CA2DB0A48AA2073B9
:1042380000E08F902020FACE209ECD20FDCE208F4A
:10424800CD68AAA56548A564488A48209ED768A86D
:104258008A484CD6CF20F1CE68A8B9EABF8555B9AF
:10426800EBBF85562054004C8DCDA0FF2CA00084B8
:104278000B20BFD1A564450B8507A565450B8508AF
:1042880020FCDB20BFD1A565450B2508450BA8A55B
:1042980064450B2507450B4C91D32090CDB013A551
:1042A8006E097F256A856AA969A000205BDCAA4C93
:1042B80061D0A900850DC64D20A6D6856186628489
:1042C80063A56CA46D20AAD6866C846DAA38E561B6
:1042D800F008A9019004A661A9FF8566A0FFE8C8B7
:1042E800CAD007A666300F18900CB16CD162F0EFF7
:1042F800A2FFB002A201E88A2A2512F002A9FF4C07
:104308003CDC20FDCEAA2090D0207900D0F460A219
:1043180000207900860C85452079002013D1B00350
:104328004C08CFA200860D860E207300900520133E
:10433800D1900BAA20730090FB2013D1B0F6C924AA
:10434800D006A9FF850DD010C925D013A510D0D04F
:10435800A980850E054585458A0980AA20730086AF
:1043680046380510E928D0034CD1D1A0008410A507
:104378002DA62E8660855FE430D004C52FF022A5D7
:1043880045D15FD008A546C8D15FF07D8818A55FE4
:10439800690790E1E8D0DCC9419005E95B38E9A5F7
:1043A800606848C92AD005A913A0DF60A545A446BE
:1043B800C954D00BC0C9F0EFC049D0034C08CFC9CD
:1043C80053D004C054F0F5A52FA430855F8460A5B0
:1043D80031A432855A845B1869079001C8855884CE
:1043E8005920B8C3A558A459C8852F8430A000A562
:1043F80045915FC8A546915FA900C8915FC8915FC4
:10440800C8915FC8915FC8915FA55F186902A460F1
:104418009001C88547844860A50B0A6905655FA4B3
:10442800609001C88558845960908000000020BFC2
:10443800D1A564A46560207300209ECD208DCDA5F4
:1044480066300DA561C9909009A9A5A0D1205BDCB3
:10445800D07A4C9BDCA50C050E48A50D48A0009809
:1044680048A54648A5454820B2D16885456885468F
:1044780068A8BABD020148BD010148A5649D0201B2
:10448800A5659D0101C8207900C92CF0D2840B20B4
:10449800F7CE68850D68850E297F850CA62FA53077
:1044A800865F8560C532D004E431F039A000B15F81
:1044B800C8C545D006A546D15FF016C8B15F1865D6
:1044C8005FAAC8B15F656090D7A2122CA20E4C37C4
:1044D800C4A213A50CD0F72094D1A50BA004D15FDA
:1044E800D0E74CEAD22094D12008C4A0008472A25C
:1044F80005A545915F1001CAC8A546915F1002CA7B
:10450800CA8671A50BC8C8C8915FA20BA900240C64
:10451800500868186901AA686900C8915FC88A913B
:104528005F204CD386718572A422C60BD0DC6559F6
:10453800B05D8559A88A65589003C8F0522008C410
:1045480085318432A900E672A471F005889158D0AB
:10455800FBC659C672D0F5E65938A531E55FA00209
:10456800915FA532C8E560915FA50CD062C8B15FC4
:10457800850BA90085718572C868AA8564688565F8
:10458800D15F900ED006C88AD15F90074C45D24CB7
:1045980035C4C8A572057118F00A204CD38A656421
:1045A800AA98A42265658671C60BD0CA8572A20531
:1045B800A5451001CAA5461002CACA8628A9002026
:1045C80055D38A655885479865598548A8A5476091
:1045D8008422B15F852888B15F8529A910855DA2ED
:1045E80000A0008A0AAA982AA8B0A4067126729088
:1045F8000B188A6528AA986529A8B093C65DD0E3E8
:1046080060A50DF00320A6D62026D538A533E531C0
:10461800A8A534E532A200860D85628463A2904C79
:1046280044DC3820F0FFA900F0EBA63AE8D0A0A2BD
:10463800152CA21B4C37C420E1D320A6D320FACED8
:10464800A9808510208BD0208DCD20F7CEA9B2204F
:10465800FFCE48A54848A54748A57B48A57A4820E5
:10466800F8C84C4FD4A9A520FFCE09808510209208
:10467800D0854E844F4C8DCD20E1D3A54F48A54E13
:104688004820F1CE208DCD68854E68854FA002B1B7
:104698004E8547AAC8B14EF0998548C8B1474888A1
:1046A80010FAA44820D4DBA57B48A57A48B14E85EA
:1046B8007AC8B14E857BA54848A54748208ACD6869
:1046C800854E68854F207900F0034C08CF68857ABD
:1046D80068857BA00068914E68C8914E68C8914E65
:1046E80068C8914E68C8914E60208DCDA00020DF2B
:1046F800DD6868A9FFA000F012A664A4658650844E
:104708005120F4D486628463856160A2228607867C
:1047180008856F847085628463A0FFC8B16FF00C50
:10472800C507F004C508D0F3C922F00118846198C0
:10473800656F8571A6709001E88672A570F004C94E
:1047480002D00B982075D4A66FA4702088D6A61620
:10475800E022D005A2194C37C4A5619500A5629541
:1047680001A5639502A00086648465847088840D21
:104778008617E8E8E8861660460F4849FF3865332B
:10478800A434B00188C4329011D004C531900B858F
:1047980033843485358436AA6860A210A50F30B6F4
:1047A8002026D5A980850F68D0D0A637A5388633AE
:1047B8008534A000844F844EA531A632855F86607B
:1047C800A919A20085228623C516F00520C7D5F0B1
:1047D800F7A9078553A52DA62E85228623E430D078
:1047E80004C52FF00520BDD5F0F385588659A903D7
:1047F8008553A558A659E432D007C531D0034C06D5
:10480800D685228623A000B122AAC8B12208C8B141
:104818002265588558C8B122655985592810D38A08
:1048280030D0C8B122A0000A69056522852290020D
:10483800E623A623E459D004C558F0BA20C7D5F01A
:10484800F3B1223035C8B1221030C8B122F02BC8DC
:10485800B122AAC8B122C5349006D01EE433B01ADA
:10486800C5609016D004E45F9010865F8560A5222D
:10487800A623854E864FA5538555A55318652285D1
:10488800229002E623A623A00060A54F054EF0F56E
:10489800A55529044AA88555B14E655F855AA56076
:1048A8006900855BA533A6348558865920BFC3A403
:1048B80055C8A558914EAAE659A559C8914E4C2AF3
:1048C800D5A56548A564482083CE208FCD68856F1F
:1048D800688570A000B16F1871649005A2174C37F5
:1048E800C42075D4207AD6A550A45120AAD6208CED
:1048F800D6A56FA47020AAD620CAD44CB8CDA000E3
:10490800B16F48C8B16FAAC8B16FA868862284235E
:10491800A8F00A4888B122913598D0F8681865350A
:1049280085359002E63660208FCDA564A465852282
:10493800842320DBD608A000B12248C8B122AAC827
:10494800B122A86828D013C434D00FE433D00B4860
:1049580018653385339002E634688622842360C460
:1049680018D00CC517D0088516E9038517A0006074
:1049780020A1D78A48A901207DD468A00091626847
:10498800684CCAD42061D7D150989004B150AA98E5
:10499800488A48207DD4A550A45120AAD668A86882
:1049A80018652285229002E62398208CD64CCAD41A
:1049B8002061D718F15049FF4C06D7A9FF8565201B
:1049C8007900C929F00620FDCE209ED72061D7F0B6
:1049D8004BCA8A4818A200F150B0B649FFC5659085
:1049E800B1A565B0AD20F7CE68A868855568686838
:1049F800AA688550688551A555489848A0008A60DE
:104A08002082D74CA2D320A3D6A200860DA860206E
:104A180082D7F008A000B122A84CA2D34C48D220DB
:104A28007300208ACD20B8D1A664D0F0A6654C7951
:104A3800002082D7D0034CF7D8A67AA47B8671844D
:104A480072A622867A1865228524A623867B900181
:104A5800E88625A000B1244898912420790020F305
:104A6800DC68A0009124A671A472867A847B6020F9
:104A78008ACD20F7D720FDCE4C9ED7A566309DA5C0
:104A880061C991B097209BDCA564A4658414851541
:104A980060A51548A5144820F7D7A000B114A86848
:104AA80085146885154CA2D320EBD78AA0009114F1
:104AB8006020EBD78649A200207900F00320F1D7C7
:104AC800864AA000B114454A2549F0F860A911A00A
:104AD800DF4C67D8208CDAA56649FF8566456E8568
:104AE8006FA5614C6AD82099D9903C208CDAD00304
:104AF8004CFCDBA6708656A269A569A8F0CE38E5FD
:104B080061F02490128461A46E846649FF6900A054
:104B1800008456A261D004A0008470C9F930C7A8E7
:104B2800A570560120B0D9246F1057A061E069F034
:104B380002A0693849FF65568570B90400F50485F7
:104B480065B90300F5038564B90200F5028563B908
:104B58000100F5018562B0032047D9A0009818A686
:104B680062D04AA6638662A6648663A6658664A642
:104B780070866584706908C920D0E4A900856185BC
:104B8800666065568570A565656D8565A564656C07
:104B98008564A563656B8563A562656A85624C3625
:104BA800D969010670266526642663266210F238E4
:104BB800E561B0C749FF69018561900EE661F04281
:104BC8006662666366646665667060A56649FF85A9
:104BD80066A56249FF8562A56349FF8563A56449A7
:104BE800FF8564A56549FF8565A57049FF8570E661
:104BF80070D00EE665D00AE664D006E663D002E619
:104C08006260A20F4C37C4A225B4048470B4039424
:104C180004B4029403B4019402A4689401690830AE
:104C2800E8F0E6E908A8A570B01416019002F601AC
:104C3800760176017602760376046AC8D0EC1860AD
:104C48008100000000037F5E56CB7980139B0B64C4
:104C580080763893168238AA3B20803504F3348155
:104C68003504F334808000000080317217F8202B5F
:104C7800DCF00210034C48D2A561E97F48A9808581
:104C880061A9D6A0D92067D8A9DBA0D9200FDBA9B4
:104C9800BCA0D92050D8A9C1A0D92040E0A9E0A043
:104CA800D92067D868207EDDA9E5A0D9208CDAD084
:104CB800034C8BDA20B7DAA9008526852785288555
:104CC80029A5702059DAA5652059DAA5642059DA92
:104CD800A5632059DAA562205EDA4C8FDBD0034C3D
:104CE80083D94A0980A8901918A529656D8529A531
:104CF80028656C8528A527656B8527A526656A859F
:104D08002666266627662866296670984AD0D66081
:104D180085228423A004B122856D88B122856C8800
:104D2800B122856B88B122856E4566856FA56E09AF
:104D380080856A88B1228569A56160A569F01F1818
:104D480065619004301D182C101469808561D003AA
:104D58004CFBD8A56F856660A56649FF3005686875
:104D68004CF7D84C7ED9200CDCAAF010186902B098
:104D7800F2A200866F2077D8E661F0E76084200011
:104D88000000200CDCA9F9A0DAA200866F20A2DBC3
:104D98004C12DB208CDAF076201BDCA90038E561A8
:104DA800856120B7DAE661F0BAA2FCA901A46AC459
:104DB80062D010A46BC463D00AA46CC464D004A4E9
:104DC8006DC465082A9009E89529F0321034A901C4
:104DD80028B00E066D266C266B266AB0E630CE101B
:104DE800E2A8A56DE565856DA56CE564856CA56B88
:104DF800E563856BA56AE562856A984C4FDBA94037
:104E0800D0CE0A0A0A0A0A0A8570284C8FDBA21437
:104E18004C37C4A5268562A5278563A5288564A582
:104E28002985654CD7D885228423A004B1228565BD
:104E380088B122856488B122856388B12285660994
:104E480080856288B1228561847060A25C2CA2573B
:104E5800A000F004A649A44A201BDC86228423A0D3
:104E680004A565912288A564912288A5639122886A
:104E7800A566097F2562912288A5619122847060C8
:104E8800A56E8566A205B5689560CAD0F98670607A
:104E9800201BDCA206B5609568CAD0F9867060A5AB
:104EA80061F0FB067090F7206FD9D0F24C38D9A585
:104EB80061F009A5662AA9FFB002A90160202BDCD0
:104EC8008562A9008563A288A56249FF2AA9008591
:104ED8006585648661857085664CD2D8466660852E
:104EE800248425A000B124C8AAF0C4B124456630A2
:104EF800C2E461D021B1240980C562D019C8B124A7
:104F0800C563D012C8B124C564D00BC8A97FC570C9
:104F1800B124E565F028A566900249FF4C31DCA56F
:104F280061F04A38E9A024661009AAA9FF8568201B
:104F38004DD98AA261C9F910062099D9846860A858
:104F4800A566298046620562856220B0D9846860BA
:104F5800A561C9A0B020209BDC8470A56684664941
:104F6800802AA9A08561A56585074CD2D885628568
:104F78006385648565A860A000A20A945DCA10FBD9
:104F8800900FC92DD0048667F004C92BD005207373
:104F980000905BC92EF02EC945D0302073009017C1
:104FA800C9ABF00EC92DF00AC9AAF008C92BF00444
:104FB800D0076660207300905C2460100EA900384A
:104FC800E55E4C49DD665F245F50C3A55E38E55D4C
:104FD800855EF012100920FEDAE65ED0F9F00720AF
:104FE800E2DAC65ED0F9A5673001604CB4DF482428
:104FF8005F1002E65D20E2DA6838E930207EDD4C99
:105008000ADD48200CDC68203CDCA56E4566856F0F
:10501800A6614C6AD8A55EC90A9009A964246030C3
:10502800114C7ED90A0A18655E0A18A000717A38F0
:10503800E930855E4C30DD9B3EBC1FFD9E6E6B27C4
:10504800FD9E6E6B2800A971A0C320DADDA53AA6E3
:105058003985628663A290382049DC20DFDD4C1E4A
:10506800CBA001A92024661002A92D99FF0085660E
:105078008471C8A930A661D0034C04DFA900E08080
:10508800F002B009A9BDA0DD2028DAA9F7855DA93D
:10509800B8A0DD205BDCF01E1012A9B3A0DD205BF8
:1050A800DCF002100E20E2DAC65DD0EE20FEDAE671
:1050B8005DD0DC2049D8209BDCA201A55D18690AD7
:1050C8003009C90BB00669FFAAA90238E902855E52
:1050D800865D8AF0021013A471A92EC899FF008A70
:1050E800F006A930C899FF008471A000A280A565C8
:1050F800187919DF8565A5647918DF8564A5637952
:1051080017DF8563A5627916DF8562E8B00410DED3
:10511800300230DA8A900449FF690A692FC8C8C882
:10512800C88447A471C8AA297F99FF00C65DD00624
:10513800A92EC899FF008471A4478A49FF2980AA2B
:10514800C024F004C03CD0A6A471B9FF0088C930BF
:10515800F0F8C92EF001C8A92BA65EF02E1008A9F8
:105168000038E55EAAA92D990101A9459900018A8F
:10517800A22F38E8E90AB0FB693A9903018A990233
:1051880001A900990401F00899FF00A900990001FC
:10519800A900A001608000000000FA0A1F00009822
:1051A8009680FFF0BDC0000186A0FFFFD8F0000088
:1051B80003E8FFFFFF9C0000000AFFFFFFFFFFDF7F
:1051C8000A8000034BC0FFFF736000000E10FFFF52
:1051D800FDA80000003CBFAAAAAAAAAAAAAAAAAA2D
:1051E800AAAAAAAAAAAAAAAAAAAAAAAAAAAAAAAA17
:1051F800AAAAAAAAAA200CDCA911A0DF20A2DBF087
:1052080070A569D0034CF9D8A24EA00020D4DBA524
:105218006E100F20CCDCA94EA000205BDCD00398D8
:10522800A40720FEDB984820EAD9A94EA000202830
:10523800DA20EDDF684A900AA561F006A56649FF05
:105248008566608138AA3B29077134583E56741622
:105258007EB31B772FEEE3857A1D841C2A7C635965
:10526800580A7E75FDE7C68031721810810000006B
:1052780000A9BFA0DF2028DAA57069509003202379
:10528800DC8556201C224A564C201E001824427EDB
:10529800424242007C22223C22227C001C224040C6
:1052A80040221C0078242222222478007E40407864
:1052B80040407E007E404078404040001C22404EE6
:1052C80042221C004242427E424242001C08080818
:1052D80008081C000E0404040444380042444870C2
:1052E800484442004040404040407E0042665A5A8E
:1052F800424242004262524A464242001824424216
:10530800422418007C42427C40404000182442421B
:105318004A241A007C42427C484442003C42403CB9
:1053280002423C003E08080808080800424242427F
:1053380042423C0042424224241818004242425A47
:105348005A66420042422418244242002222221C69
:10535800080808007E02041820407E003C20202017
:1053680020203C000C10103C10706E003C0404041B
:1053780004043C0000081C2A080808080000102043
:105388007F20100000000000000000000808080846
:1053980000000800242424000000000024247E24A7
:1053A8007E242400081E281C0A3C080000626408A9
:1053B80010264600304848304A443A000408100095
:1053C800000000000408101010080400201008084D
:1053D80008102000082A1C3E1C2A08000008083E65
:1053E8000808000000000000000808100000007E07
:1053F8000000000000000000001818000002040867
:10540800102040003C42465A62423C0008182808D6
:1054180008083E003C42020C30407E003C42021C20
:1054280002423C00040C14247E0404007E407804EC
:10543800024438001C20407C42423C007E42040862
:10544800101010003C42423C42423C003C42423E6A
:1054580002043800000008000008000000000800EE
:10546800000808100E18306030180E0000007E008A
:105478007E00000070180C060C1870003C42020CEC
:105488001000100000000000FF000000081C3E7F14
:105498007F1C3E001010101010101010000000FFAC
:1054A800000000000000FF000000000000FF0000F6
:1054B800000000000000000000FF00002020202065
:1054C8002020202004040404040404040000000034
:1054D800E01008080808080403000000080808107D
:1054E800E000000080808080808080FF8040201065
:1054F800080402010102040810204080FF80808017
:1055080080808080FF01010101010101003C7E7E55
:105518007E7E3C00000000000000FF00367F7F7F99
:105528003E1C080040404040404040400000000011
:10553800030408088142241818244281003C42428E
:1055480042423C00081C2A772A080800020202028C
:1055580002020202081C3E7F3E1C080008080808D8
:10556800FF080808A050A050A050A050080808083C
:10557800080808080000013E54141400FF7F3F1F6C
:105588000F0703010000000000000000F0F0F0F039
:10559800F0F0F0F000000000FFFFFFFFFF00000048
:1055A8000000000000000000000000FF80808080F4
:1055B80080808080AA55AA55AA55AA5501010101E3
:1055C8000101010100000000AA55AA55FFFEFCF8E0
:1055D800F0E0C0800303030303030303080808087B
:1055E8000F080808000000000F0F0F0F0808080830
:1055F8000F00000000000000F80808080000000084
:105608000000FFFF000000000F080808080808084D
:10561800FF00000000000000FF080808080808084C
:10562800F8080808C0C0C0C0C0C0C0C0E0E0E0E0E2
:10563800E0E0E0E00707070707070707FFFF0000AC
:1056480000000000FFFFFF00000000000000000055
:1056580000FFFFFF01010101010101FF000000003F
:10566800F0F0F0F00F0F0F0F000000000808080816
:10567800F8000000F0F0F0F000000000F0F0F0F0AA
:105688000F0F0F0FE3DDB5A9B3DFE1FFE7DBBD8146
:10569800BDBDBDFF83DDDDC3DDDD83FFE3DDBFBF52
:1056A800BFDDE3FF87DBDDDDDDDB87FF81BFBF8794
:1056B800BFBF81FF81BFBF87BFBFBFFFE3DDBFB1F2
:1056C800BDDDE3FFBDBDBD81BDBDBDFFE3F7F7F7A0
:1056D800F7F7E3FFF1FBFBFBFBBBC7FFBDBBB78FD6
:1056E800B7BBBDFFBFBFBFBFBFBF81FFBD99A5A5EA
:1056F800BDBDBDFFBD9DADB5B9BDBDFFE7DBBDBD42
:10570800BDDBE7FF83BDBD83BFBFBFFFE7DBBDBD1B
:10571800B5DBE5FF83BDBD83B7BBBDFFC3BDBFC35D
:10572800FDBDC3FFC1F7F7F7F7F7F7FFBDBDBDBD77
:10573800BDBDC3FFBDBDBDDBDBE7E7FFBDBDBDA58F
:10574800A599BDFFBDBDDBE7DBBDBDFFDDDDDDE34D
:10575800F7F7F7FF81FDFBE7DFBF81FFC3DFDFDF7F
:10576800DFDFC3FFF3EFEFC3EF8F91FFC3FBFBFB5B
:10577800FBFBC3FFFFF7E3D5F7F7F7F7FFFFEFDF13
:1057880080DFEFFFFFFFFFFFFFFFFFFFF7F7F7F7F0
:10579800FFFFF7FFDBDBDBFFFFFFFFFFDBDB81DB6F
:1057A80081DBDBFFF7E1D7E3F5C3F7FFFF9D9BF74D
:1057B800EFD9B9FFCFB7B7CFB5BBC5FFFBF7EFFF41
:1057C800FFFFFFFFFBF7EFEFEFF7FBFFDFEFF7F769
:1057D800F7EFDFFFF7D5E3C1E3D5F7FFFFF7F7C131
:1057E800F7F7FFFFFFFFFFFFFFF7F7EFFFFFFF816F
:1057F800FFFFFFFFFFFFFFFFFFE7E7FFFFFDFBF7EF
:10580800EFDFBFFFC3BDB9A59DBDC3FFF7E7D7F75E
:10581800F7F7C1FFC3BDFDF3CFBF81FFC3BDFDE3F4
:10582800FDBDC3FFFBF3EBDB81FBFBFF81BF87FB08
:10583800FDBBC7FFE3DFBF83BDBDC3FF81BDFBF772
:10584800EFEFEFFFC3BDBDC3BDBDC3FFC3BDBDC14A
:10585800FDFBC7FFFFFFF7FFFFF7FFFFFFFFF7FFA6
:10586800FFF7F7EFF1E7CF9FCFE7F1FFFFFF81FFEA
:1058780081FFFFFF8FE7F3F9F3E78FFFC3BDFDF368
:10588800EFFFEFFFFFFFFFFF00FFFFFFF7E3C18020
:1058980080E3C1FFEFEFEFEFEFEFEFEFFFFFFF0068
:1058A800FFFFFFFFFFFF00FFFFFFFFFFFF00FFFFFE
:1058B800FFFFFFFFFFFFFFFFFF00FFFFDFDFDFDF6F
:1058C800DFDFDFDFFBFBFBFBFBFBFBFBFFFFFFFF80
:1058D8001FEFF7F7F7F7F7FBFCFFFFFFF7F7F7EF17
:1058E8001FFFFFFF7F7F7F7F7F7F7F007FBFDFEF0F
:1058F800F7FBFDFEFEFDFBF7EFDFBF7F007F7F7F3D
:105908007F7F7F7F00FEFEFEFEFEFEFEFFC38181DD
:105918008181C3FFFFFFFFFFFFFF00FFC980808079
:10592800C1E3F7FFBFBFBFBFBFBFBFBFFFFFFFFFE1
:10593800FCFBF7F77EBDDBE7E7DBBD7EFFC3BDBD44
:10594800BDBDC3FFF7E3D588D5F7F7FFFDFDFDFD26
:10595800FDFDFDFDF7E3C180C1E3F7FFF7F7F7F7BA
:1059680000F7F7F75FAF5FAF5FAF5FAFF7F7F7F736
:10597800F7F7F7F7FFFFFEC1ABEBEBFF0080C0E0E6
:10598800F0F8FCFEFFFFFFFFFFFFFFFF0F0F0F0FF9
:105998000F0F0F0FFFFFFFFF0000000000FFFFFFCA
:1059A800FFFFFFFFFFFFFFFFFFFFFF007F7F7F7FFE
:1059B8007F7F7F7F55AA55AA55AA55AAFEFEFEFEEF
:1059C800FEFEFEFEFFFFFFFF55AA55AA00010307D2
:1059D8000F1F3F7FFCFCFCFCFCFCFCFCF7F7F7F717
:1059E800F0F7F7F7FFFFFFFFF0F0F0F0F7F7F7F742
:1059F800F0FFFFFFFFFFFFFF07F7F7F7FFFFFFFFCE
:105A0800FFFF0000FFFFFFFFF0F7F7F7F7F7F7F7E3
:105A180000FFFFFFFFFFFFFF00F7F7F7F7F7F7F7C4
:105A280007F7F7F73F3F3F3F3F3F3F3F1F1F1F1F0E
:105A38001F1F1F1FF8F8F8F8F8F8F8F80000FFFF24
:105A4800FFFFFFFF000000FFFFFFFFFFFFFFFFFF5B
:105A5800FF000000FEFEFEFEFEFEFE00FFFFFFFF51
:105A68000F0F0F0FF0F0F0F0FFFFFFFFF7F7F7F75A
:105A780007FFFFFF0F0F0F0FFFFFFFFF0F0F0F0FA6
:105A8800F0F0F0F01C224A564C201E0000003804AA
:105A98003C443A0040405C6242625C0000003C4288
:105AA80040423C0002023A4642463A0000003C426C
:105AB8007E403C000C12107C1010100000003A468A
:105AC800463A023C40405C624242420008001808E4
:105AD80008081C0004000C040404443840404448EE
:105AE800506844001808080808081C000000764997
:105AF8004949490000005C624242420000003C42C1
:105B080042423C0000005C62625C404000003A4651
:105B1800463A020200005C624040400000003E40FD
:105B28003C027C0010107C1010120C000000424255
:105B380042463A000000424242241800000041490F
:105B4800494936000000422418244200000042421D
:105B5800463A023C00007E0418207E003C202020AB
:105B680020203C000C10103C10706E003C04040413
:105B780004043C0000081C2A08080808000010203B
:105B88007F2010000000000000000000080808083E
:105B980000000800242424000000000024247E249F
:105BA8007E242400081E281C0A3C080000626408A1
:105BB80010264600304848304A443A00040810008D
:105BC8000000000004081010100804002010080845
:105BD80008102000082A1C3E1C2A08000008083E5D
:105BE8000808000000000000000808100000007EFF
:105BF800000000000000000000181800000204085F
:105C0800102040003C42465A62423C0008182808CE
:105C180008083E003C42020C30407E003C42021C18
:105C280002423C00040C14247E0404007E407804E4
:105C3800024438001C20407C42423C007E4204085A
:105C4800101010003C42423C42423C003C42423E62
:105C580002043800000008000008000000000800E6
:105C6800000808100E18306030180E0000007E0082
:105C78007E00000070180C060C1870003C42020CE4
:105C88001000100000000000FF0000001824427EF1
:105C9800424242007C22223C22227C001C224040BC
:105CA80040221C0078242222222478007E4040785A
:105CB80040407E007E404078404040001C22404EDC
:105CC80042221C004242427E424242001C0808080E
:105CD80008081C000E0404040444380042444870B8
:105CE800484442004040404040407E0042665A5A84
:105CF800424242004262524A46424200182442420C
:105D0800422418007C42427C404040001824424211
:105D18004A241A007C42427C484442003C42403CAF
:105D280002423C003E080808080808004242424275
:105D380042423C0042424224241818004242425A3D
:105D48005A66420042422418244242002222221C5F
:105D5800080808007E02041820407E000808080889
:105D6800FF080808A050A050A050A0500808080834
:105D780008080808CCCC3333CCCC3333CC66339901
:105D8800CC6633990000000000000000F0F0F0F04D
:105D9800F0F0F0F000000000FFFFFFFFFF00000040
:105DA8000000000000000000000000FF80808080EC
:105DB80080808080AA55AA55AA55AA5501010101DB
:105DC8000101010100000000AA55AA55993366CCCB
:105DD800993366CC03030303030303030808080885
:105DE8000F080808000000000F0F0F0F0808080828
:105DF8000F00000000000000F8080808000000007C
:105E08000000FFFF000000000F0808080808080845
:105E1800FF00000000000000FF0808080808080844
:105E2800F8080808C0C0C0C0C0C0C0C0E0E0E0E0DA
:105E3800E0E0E0E00707070707070707FFFF0000A4
:105E480000000000FFFFFF0000000000000000004D
:105E580000FFFFFF010244485060400000000000BE
:105E6800F0F0F0F00F0F0F0F00000000080808080E
:105E7800F8000000F0F0F0F000000000F0F0F0F0A2
:105E88000F0F0F0FE3DDB5A9B3DFE1FFFFFFC7FB7E
:105E9800C3BBC5FFBFBFA39DBD9DA3FFFFFFC3BD80
:105EA800BFBDC3FFFDFDC5B9BDB9C5FFFFFFC3BD7C
:105EB80081BFC3FFF3EDEF83EFEFEFFFFFFFC5B93E
:105EC800B9C5FDC3BFBFA39DBDBDBDFFF7FFE7F7C4
:105ED800F7F7E3FFFBFFF3FBFBFBBBC7BFBFBBB79A
:105EE800AF97BBFFE7F7F7F7F7F7E3FFFFFF89B6D1
:105EF800B6B6B6FFFFFFA39DBDBDBDFFFFFFC3BD87
:105F0800BDBDC3FFFFFFA39D9DA3BFBFFFFFC5B9D5
:105F1800B9C5FDFDFFFFA39DBFBFBFFFFFFFC1BF09
:105F2800C3FD83FFEFEF83EFEFEDF3FFFFFFBDBD91
:105F3800BDB9C5FFFFFFBDBDBDDBE7FFFFFFBEB6B7
:105F4800B6B6C9FFFFFFBDDBE7DBBDFFFFFFBDBD89
:105F5800B9C5FDC3FFFF81FBE7DF81FFC3DFDFDFDB
:105F6800DFDFC3FFF3EFEFC3EF8F91FFC3FBFBFB53
:105F7800FBFBC3FFFFF7E3D5F7F7F7F7FFFFEFDF0B
:105F880080DFEFFFFFFFFFFFFFFFFFFFF7F7F7F7E8
:105F9800FFFFF7FFDBDBDBFFFFFFFFFFDBDB81DB67
:105FA80081DBDBFFF7E1D7E3F5C3F7FFFF9D9BF745
:105FB800EFD9B9FFCFB7B7CFB5BBC5FFFBF7EFFF39
:105FC800FFFFFFFFFBF7EFEFEFF7FBFFDFEFF7F761
:105FD800F7EFDFFFF7D5E3C1E3D5F7FFFFF7F7C129
:105FE800F7F7FFFFFFFFFFFFFFF7F7EFFFFFFF8167
:105FF800FFFFFFFFFFFFFFFFFFE7E7FFFFFDFBF7E7
:10600800EFDFBFFFC3BDB9A59DBDC3FFF7E7D7F756
:10601800F7F7C1FFC3BDFDF3CFBF81FFC3BDFDE3EC
:10602800FDBDC3FFFBF3EBDB81FBFBFF81BF87FB00
:10603800FDBBC7FFE3DFBF83BDBDC3FF81BDFBF76A
:10604800EFEFEFFFC3BDBDC3BDBDC3FFC3BDBDC142
:10605800FDFBC7FFFFFFF7FFFFF7FFFFFFFFF7FF9E
:10606800FFF7F7EFF1E7CF9FCFE7F1FFFFFF81FFE2
:1060780081FFFFFF8FE7F3F9F3E78FFFC3BDFDF360
:10608800EFFFEFFFFFFFFFFF00FFFFFFE7DBBD8133
:10609800BDBDBDFF83DDDDC3DDDD83FFE3DDBFBF48
:1060A800BFDDE3FF87DBDDDDDDDB87FF81BFBF878A
:1060B800BFBF81FF81BFBF87BFBFBFFFE3DDBFB1E8
:1060C800BDDDE3FFBDBDBD81BDBDBDFFE3F7F7F796
:1060D800F7F7E3FFF1FBFBFBFBBBC7FFBDBBB78FCC
:1060E800B7BBBDFFBFBFBFBFBFBF81FFBD99A5A5E0
:1060F800BDBDBDFFBD9DADB5B9BDBDFFE7DBBDBD38
:10610800BDDBE7FF83BDBD83BFBFBFFFE7DBBDBD11
:10611800B5DBE5FF83BDBD83B7BBBDFFC3BDBFC353
:10612800FDBDC3FFC1F7F7F7F7F7F7FFBDBDBDBD6D
:10613800BDBDC3FFBDBDBDDBDBE7E7FFBDBDBDA585
:10614800A599BDFFBDBDDBE7DBBDBDFFDDDDDDE343
:10615800F7F7F7FF81FDFBE7DFBF81FFF7F7F7F7F9
:1061680000F7F7F75FAF5FAF5FAF5FAFF7F7F7F72E
:10617800F7F7F7F73333CCCC3333CCCC3399CC6641
:106188003399CC66FFFFFFFFFFFFFFFF0F0F0F0FD5
:106198000F0F0F0FFFFFFFFF0000000000FFFFFFC2
:1061A800FFFFFFFFFFFFFFFFFFFFFF007F7F7F7FF6
:1061B8007F7F7F7F55AA55AA55AA55AAFEFEFEFEE7
:1061C800FEFEFEFEFFFFFFFF55AA55AA66CC9933D7
:1061D80066CC9933FCFCFCFCFCFCFCFCF7F7F7F7FD
:1061E800F0F7F7F7FFFFFFFFF0F0F0F0F7F7F7F73A
:1061F800F0FFFFFFFFFFFFFF07F7F7F7FFFFFFFFC6
:10620800FFFF0000FFFFFFFFF0F7F7F7F7F7F7F7DB
:1062180000FFFFFFFFFFFFFF00F7F7F7F7F7F7F7BC
:1062280007F7F7F73F3F3F3F3F3F3F3F1F1F1F1F06
:106238001F1F1F1FF8F8F8F8F8F8F8F80000FFFF1C
:10624800FFFFFFFF000000FFFFFFFFFFFFFFFFFF53
:10625800FF000000FEFDBBB7AF9FBFFFFFFFFFFFC2
:106268000F0F0F0FF0F0F0F0FFFFFFFFF7F7F7F752
:1062780007FFFFFF0F0F0F0FFFFFFFFF0F0F0F0F9E
:10628800F0F0F0F000000000000000000000000046
:1062980000000000000000000000000000000000F6
:1062A80000000000000000000000000000000000E6
:1062B80000000000000000000000000000000000D6
:1062C80000000000000000000000000000000000C6
:0482880000000000F2
:00000001FF
